:020000022000DC
:1000000000400020C50102000502020007020200B4
:1000100000000000000000000000000000000000E0
:1000200000000000000000000000000009020200C3
:1000300000000000000000000B0202000D020200A0
:100040001102020013020200150202001702020050
:100050001902020000000000391D0200C11A02004E
:100060001F02020021020200E52202002502020016
:1000700027020200290202002B0202002D020200C8
:100080002F0202009147020033020200000000002C
:100090005948020037020200993F02003B02020069
:1000A0003D0202003F0202000000000000000000CC
:1000B0000000000000000000000000000000000040
:1000C000164B002B00D1144B9D46402292029A1AE7
:1000D000924600218B460F461348144A121A00F02C
:1000E00067F80F4B002B00D098470E4B002B00D029
:1000F00098470020002104000D000D48002802D080
:100100000C4800E000BF00F02DF82000290001F0AD
:1001100007FB00F011F8C046000008000040002076
:100120000000000000000000382600206C2F002096
:100130000000000000000000084B10B5041C002B5C
:1001400002D0002100E000BF054B1868836A002B35
:1001500000D09847201C00F033F8C0460000000093
:1001600090B0020070B50E4B0E4D0024ED1AAD108C
:100170001E1CAC4204D0A300F35898470134F8E7A2
:100180000AF078FF084B094D0024ED1AAD101E1C33
:10019000AC4204D0A300F35898470134F8E770BD8F
:1001A000B0240020B0240020B0240020B02400207F
:1001B000031C8218934202D019700133FAE770478A
:1001C000FEE7C0460948026803210A430260084965
:1001D000084A094B9B1A05DD0024085910510434C4
:1001E0009C42FADB0548804705480047240500404B
:1001F000B4B4020000240020B02400204102020018
:10020000C1000200FEE7FEE7FEE7FEE7FEE7FEE7CD
:10021000FEE7FEE7FEE7FEE7FEE7FEE7FEE7FEE7B6
:10022000FEE7FEE7FEE7FEE7FEE7FEE7FEE7FEE7A6
:10023000FEE7FEE7FEE7FEE7FEE7FEE7FEE7FEE796
:100240001C4B10B51A78181C012A12D11A4B1B68C6
:1002500019070ED1194BF0221B68E024191C11401C
:10026000234204D1164B1B68134202D118E03029F7
:10027000F8D00378012B1BD10F4A1268110717D150
:100280000E4A1168F0221140402911D10C49096829
:1002900011420DD1C1228021D200C9058B5007E047
:1002A0000849094A11608021084A09021160E0E703
:1002B00010BDC046E00F00F0E40F00F0E80F00F0C2
:1002C000EC0F00F0DFFF07C004050040186C004091
:1002D00073DF704776DF704778DF70477ADF7047EB
:1002E0007CDF70477FDF704781DF7047A9DF704791
:1002F00008B54821FF31024A00F074FD08BDC04630
:100300009CB0020008B50378012B04D0022B04D165
:1003100003F088FA01E002F0F7FE08BD13B5041CF3
:1003200004F02CFF3B48211C03F0EFFA2388142B28
:1003300054D00ED8112B18D0132B1FD0102B68D1EE
:10034000354B00221A70354B1B681B689847A288F2
:1003500011E0192B2ED0522B36D0172B59D1A11DBD
:1003600032222F4808F06CFE53E02C4B1B685B6870
:100370009847012252422B4B1A804AE06A461E23BC
:100380001380937801221343E12213400C2213437C
:10039000202293436A4693700723D370102313716E
:1003A000204B00211888FFF79DFF002831D0402105
:1003B000FF312BE0A379002B2BD1174A1370174B79
:1003C0001B689B68984724E0164B00210A1C18887C
:1003D000FFF78CFFCD2100281BD016E01049E289E1
:1003E000C888104B904208D1063118880022FFF7C8
:1003F0007BFFD32100280CD007E0002118880A1CBD
:10040000FFF772FF002804D0D6214900064A00F009
:10041000E9FC13BD402600203C26002038260020A1
:10042000C8260020642400209CB0020008B5037890
:10043000002B0BD1064B3B211888FFF74BFF002800
:1004400004D02821FF31034A00F0CCFC08BDC0468F
:10045000642400209CB0020008B5031C0A1C02485A
:10046000191C00F0BFFC08BDEFBEADDE70B5061C68
:100470000D1C02F0D9FF041E04D0EE2149000F4AE2
:1004800000F0B0FC0E4B1A880E4B9A4205D00E4875
:10049000311C2A1C03F082FC041C0C4B9C420BD028
:1004A000112C09D00823221C9A4305D0F521201CC9
:1004B0004900024A00F096FC70BDC0469CB00200A4
:1004C00064240020FFFF00004026002003300000CD
:1004D000174A70B5136803240133051C13601C40D0
:1004E00022D1144E144B32889A421DD01348291C35
:1004F00003F018FC002817D0114A904208D1211CA3
:100500003088221CFFF7F2FE822100280CD007E081
:10051000082809D00B4A904206D0112804D0832124
:100520008900094A00F05EFC281C02F0CFFE70BD75
:10053000C426002064240020FFFF00004026002085
:1005400001340000033000009CB00200F0B59B4B6A
:1005500051221A7008229A700922FF24DA70A5B07D
:10056000051C0422181D96495C7008F069FD954B26
:1005700050221A700322DA705D221A7100225A7119
:10058000914E48229A71914852225C709C70DA71A7
:10059000356003F0E3FC002804D0E72149008C4AD1
:1005A00000F020FC8B4803F0E3FC002804D0E92194
:1005B0004900874A00F016FC874C06AD1123201C29
:1005C0002B7008F025FE211C82B2281CFFF788FE44
:1005D000002803D072217E4A00F004FC7F48FFF718
:1005E0007BFE002803D07521794A00F0FBFB14AD97
:1005F0000822281C0021FFF7DBFDC8229200C82337
:100600005B006A80281C00222B80AA80EB80FFF709
:1006100065FE002803D07F216D4A00F0E3FB06ACA5
:1006200000214022281CFFF7C3FD00211822201CB6
:10063000FFF7BEFD684B80220693694B520563604D
:100640005D232381674B68496381536E04A8A381AE
:100650000323A37370235B42E37308232374526E56
:10066000626100220093092308F0B0FD281C616834
:1006700003F0BEFE1CA804A903F0BAFE02232B81DE
:100680006B462233EB606A46042326322B820BAB87
:100690006B61EA61012310222B83134323AA137099
:1006A0006B4600228D33281C1A7003F00DFF0028C2
:1006B00003D0C421464A00F095FB14AD0C23002161
:1006C0002822281C2370FFF773FD32686C60526982
:1006D00004232A611022AB60101C012369461843D1
:1006E0005231C8770020C918C877111C19432B70E4
:1006F0001343EB776B46513329776877D877291CFA
:100700003A4803F02DF9002803D0FC21304A00F0CC
:1007100069FB306802F066FD33680220996904AE17
:1007200002F0C0FF6D4602F00BFF0623304908229D
:10073000301CEB7308F084FC0F3500213822201C9C
:10074000FFF736FDA56014AD012302270021281C08
:1007500038222770A370A38023826661FFF728FDEB
:10076000201C291C2F83EE6103F00AFE002803D011
:10077000A421174A00F036FB1C22281C0021FFF799
:1007800017FDA02292026A60AA60032200232A7346
:10079000164A14932B74174B7C3212886B61164BDC
:1007A000281CEA81AB6104F0B1FC002804D0AE2122
:1007B0004900074A00F016FB25B0F0BD602F00206D
:1007C00064000010582F0020382600201D0302006E
:1007D0009CB0020005030200A9B0020084040000DE
:1007E000B2B0020048520000BEB002004026002015
:1007F00094B002002D040200F102020010B586B090
:1008000001AC201C00211422FFF7D2FC002323702E
:100810006360237228232382201CB4236382FFF7A2
:1008200057FD002803D00649064A00F0DBFA064BC4
:1008300001221A70054B1B68DB68984706B010BD93
:10084000460200009CB002003C2600203826002012
:1008500008B5FFF7D3FF02F029FD02F0A7FE02F072
:1008600075FF08BD021C202008B5084004D00A4BC3
:100870001B685B6898470EE080235B031A4203D035
:10088000054B1B689B6805E0194204D0024B012010
:100890001B689B68984708BD1427002008B501F025
:1008A0005FFB012806D0022809D1054B01201B68F7
:1008B0001B6803E0024B00201B681B68984708BDBB
:1008C00014270020044BA022D205D05880214901D2
:1008D0004140D1507047C04604050000C3070AD507
:1008E0000C4AA0238021DB05890199508021A12297
:1008F0004901D200995083070AD5064AA0238021D6
:10090000DB05C90299508021A1220903D200995028
:100910007047C0460C050000C3070AD50C4AA02347
:100920008021DB05490199508021A1228901D20053
:10093000995083070AD5064AA0238021DB050903C5
:1009400099508021A122C902D20099507047C04617
:100950000C050000C30709D5A022A1238021D205E0
:10096000DB008901D15080214901D150830709D58D
:10097000A022A1238021D205DB00C902D150802111
:100980000903D15070470000114B10B51C680022BC
:100990000023CA030B490A48801859410A4A0B4BE5
:1009A00005F004F90022011C201C04F0B3F9002812
:1009B00004D00621FF31074A00F014FA10BDC046EA
:1009C000F401000000000000E80300000000000047
:1009D00018270020C7B00200084B10B5041C186887
:1009E00004F0E6F9002804D00E21FF31044A00F09B
:1009F000F9F9201CFFF7AEFF10BDC04618270020F4
:100A0000C7B0020038B50B4A0B4B08209C58A122F6
:100A1000D20099589D58013104F0DEFF691C041979
:100A2000102004F0D9FF011C201C04F0D5FF80B277
:100A300038BDC0460405000000100140A223A022DA
:100A4000D205DB00D35801201B0D984370470000EE
:100A500010B502F001FAA0240A4B1022E405E2507E
:100A6000094A1288510608D58022D205E250FFF7C4
:100A7000E5FF002801D101F0E7F8A1234022DB00C7
:100A8000E25010BD0C05000090FC030008B50028E2
:100A900001D000F095FFFFF7DBFF0320FFF75AFFBF
:100AA00008BD0000F8B5584B58491860A023DB0575
:100AB00001225A50E621C9005A50E921C9005A5072
:100AC0005349041C5A50E221C9005A50A121102058
:100AD000C900504D5850288846060FD54E481A5028
:100AE000EF20C0001A508022D2055A50EA2100227D
:100AF000C9005A5049495A5049495A50A023E12245
:100B0000DB050221D2009950E3220121D200995045
:100B1000E4220021D2009950C021424A8902995012
:100B20002B88590602D480277F0300E03E4F012026
:100B30003E4901F053F9002803D0A5213C4A00F0BA
:100B400051F93C4E391C301C3B4A3C4B01F082F9B8
:100B5000002803D0AB21364A00F044F9307801F088
:100B6000A5F9002803D0AE21314A00F03BF900F08E
:100B700046FF02F0ADF90320FFF7B0FE0A2004F0B3
:100B800001FF0120FFF7E6FE0220FFF7C5FEA023CC
:100B9000A122DB054021D2009950EB22D200002196
:100BA0009950C02189029950162001F0D3F9244EA2
:100BB0000121301C234A04F085F8002803D0C42109
:100BC0001B4A00F00FF930681F49002204F0A2F818
:100BD000002803D0C821164A00F004F91B4801215F
:100BE0001B4A04F06FF8002804D0A021FF31104AFE
:100BF00000F0F8F82B88E268FF2003215E0600D49D
:100C0000011C01F039F8F8BD14270020340700005A
:100C10004C07000090FC03000C07000024070000B4
:100C20002C0700001407000000021000FC26002022
:100C3000C7B002001C270020200010006508020039
:100C4000102700209D0802006606000018270020DB
:100C5000C50802002BDF70472CDF704730DF70477C
:100C600031DF704734DF704735DF704739DF704759
:100C70003DDF704711DF7047024B5970090A187049
:100C800099707047102A0020014B00221A607047AB
:100C9000542B00207047000008B500F045FF02F01B
:100CA000E5F8014B186008BDB02A00201FB5011CF3
:100CB0000822684608F0C4F96A469379022B0DD3DE
:100CC000032B01D9522B09D16946082202A808F04A
:100CD000B7F9034802A9082208F0B2F905B000BD2F
:100CE0004C2B002007B5044A00900191684608216A
:100CF00004F0BAF80EBDC046E910020008B50020A5
:100D0000011C024A04F0B0F808BDC04609110200F7
:100D100008B504F01DFC08BD38B5064D064C41234E
:100D200000202B70207001F05FFD28782178FFF7FC
:100D3000A3FF38BD132A0020142A002008B5012083
:100D4000FA218140FFF720FE08BD08B50120FFF71A
:100D500043FE08BD08B50120FFF7FCFDFFF74EFD7F
:100D600008BD08B50120FFF737FE0120FFF7D4FDCD
:100D700008BD0000F0B5002385B000930193164B29
:100D800016495A898A4225D0FA21890048431E21F2
:100D90001218181C5A81462701F072FB10266A4669
:100DA00080256B4602AC1770D670557102229A717D
:100DB00069460822201C08F043F96B46DE726B4638
:100DC00002225D736B469A730548211C0822277026
:100DD00008F036F905B0F0BD682A0020FFFF0000DA
:100DE0004C2B002070B5051C0E1C141C0320FFF7B3
:100DF00075FDB1B2221C281C01F04EF90220FFF74C
:100E000035FFFFF737FF72B6FA20800004F0BAFD15
:100E1000BFF34F8F024A034BDA60BFF34F8FFEE7F9
:100E20000400FA0500ED00E0F0B59F4B87B01A789A
:100E3000022A02D900221A70C7E09C4C2378462B64
:100E400000D0AEE0A379032B06D0522B17D1984BDC
:100E500003CB02F037F996E002F008F807F0A8FAA1
:100E6000904B8F4A06F036FC07F0FCF900B2009078
:100E7000192101200A22002302F034FB83E0E078EC
:100E800004AE02900021301C0622FFF791F902986F
:100E900010380D2877D804F095FD0B071A1E40383E
:100EA000223476767676763C8249301C02310AE02E
:100EB000804D301C291C0831022208F0C1F8291C81
:100EC00068460A311230022208F0BAF856E0794931
:100ED000301C0431F7E77749301C0631F3E701F0A5
:100EE000D7F8051C291C0222301C08F0A9F8684616
:100EF000A91C0222123008F0A3F8291D05A801221E
:100F0000E2E76C49301C1031DDE700F087FE3070FD
:100F100034E0694B1B88337030E0257904272B1CA3
:100F2000FF3B5A1E93415B421D4001F07BFC6B4628
:100F300030705D742E1CBB1EDBB203936B1CB3427E
:100F40001CDB01F06FFC864206D3039904ABFF2241
:100F50005A54791EC9B20BE0331C564A08335B0061
:100F6000D3189A88039804AB791E1A54C9B2120A8E
:100F7000013602375A54F6B2FFB2DCE762790298C2
:100F800004A902F06DFA6379802B03D07F221A4006
:100F9000012A03DC201C002108220FE0013B6371C1
:100FA0000EE0464C207800280FD0A1786378090223
:100FB0001943FFF75BFA201C00210322FFF7F8F822
:100FC00039490B7801330B7065E03D4D2B880133B7
:100FD0002B8000F0FBFF041C01F02AF8394F061C9F
:100FE0003B78A376412B02D1374B1B7805E0412B90
:100FF00004D3432B02D8354B1B8AA38301F07CFB1F
:101000002B4A231CE083283303CA03C3304B5A788E
:10101000500707D5D978621DD1771979A21DD177EC
:1010200000225A70FFF7EEFC2A4B20801B68201C20
:101030002362311C01F08CFE002801D0264907E014
:10104000201C311C04AA01F05FFA002803D02349B8
:10105000234AFFF7C7FE201CFFF73AFA3B78423BD2
:10106000DBB2012B0BD82B88D90708D400F0CAFFBC
:10107000049A3B78211C0092144A01F011FC208B49
:10108000A189400802F0A0FA164B1888431E984127
:10109000C0B202F06BFB07B0F0BDC046C046C04610
:1010A0000000000000009040F82900204C2B002098
:1010B0009C2A0020682A002090FC0300102A0020AF
:1010C000482B0020132A0020142A0020FC2900208D
:1010D000A42A0020B02A0020560200005A02000074
:1010E000DBB002004A2B002008B5031C082905D0FC
:1010F00014210020FF31034AFFF774FE40681B688B
:10110000984708BDE5B0020008B5002904D00020CA
:101110009821034AFFF766FE02F082FE08BDC04632
:1011200014B10200002008B5011C054A03F09CFE22
:10113000002804D0E821FF31024AFFF753FE08BD22
:10114000FD120200DBB0020010B5041C01F026FB0A
:10115000002807D00448211C1622123007F070FF27
:10116000FFF7E0FF10BDC046682A002070B5467842
:10117000037836021E43041C301C05F0B3FB1449EF
:1011800004F000FD00280AD0124DAB88B34206D00F
:10119000AE80FFF7C7FF281C1E2101F071F9A01CCB
:1011A00001F0D8FE051C201D01F0E2FE0021041C08
:1011B000281C04F0E7FC002801D0074B1D60201C10
:1011C000002104F0DFFC002801D0034B5C6070BDFF
:1011D0000000F041682A0020FC29002073B5C6B247
:1011E0000090301C40380C1C01911C2878D804F069
:1011F000E9FB180F242E5B64323B447777777777CF
:10120000777777777777777777777777776D7400F2
:10121000364B41221A700878354B187001F0E4FA09
:101220005EE0334B00221A70304B4022081C1A70CB
:1012300001F0ACFE01F0FCFA52E02C4B42221A7095
:101240004A780B7812021A432A4B1A8248E0274B3D
:1012500043221A7041E0254B4322081C1A7001F00A
:10126000B9FE244BD8603BE0204B4322081C1A7087
:1012700001F09EFE1F4B986032E048780B78000228
:1012800018430A2104F0A8FB1B4D83B2EA889A4256
:1012900026D0E122D200934222D9EB80FFF742FF11
:1012A000E88801F0EBFC1BE0104B4322081C1A708D
:1012B00001F050FE0F4B186012E00C4B4322081C4B
:1012C0001A7001F055FE0B4B586009E048780B7816
:1012D0000002184301F016FA02E0201CFFF746FF57
:1012E000301C2178FFF7C8FC73BDC046132A0020CC
:1012F000142A0020FC290020682A002008B505488F
:1013000001F014FE002804D0D621FF31024AFFF775
:1013100069FD08BD682A0020DBB0020073B56C4689
:101320000023073423702B4B061C5A680425D20572
:10133000D20D1FD0103AD3B259B200290CDA0F22C5
:101340001A40083A9208244992005218556803221C
:1013500013409340DD4008E08908204BC0318900EC
:10136000CD5803231A409A40D540EDB2AD09EDB2F5
:10137000012D0AD0201CFFF76DFC022801D172B6A6
:1013800003E0002801D0164906E0164B186803F068
:101390000FFD002803D01449144AFFF723FD144B16
:1013A000186803F005FDA72100280DD1301CFFF7B8
:1013B0006DFB012D0AD062B62078FFF74DFC0223A9
:1013C000021C9A4302D0EA218900E5E7FFF748FCB6
:1013D00073BDC04600ED00E018ED00E000E100E064
:1013E000A3030000AC2A002099020000DBB0020039
:1013F000B42A002037B5164B164C1A68011C083267
:1014000068461A606D4600F0BDFB231C06CD06C37E
:1014100063785B065B0F052B19D1FFF70FFB051EE9
:1014200015D1FFF779FC63781B071B0F052B0CDC2C
:101430000320FFF78FFA0220FFF750FA064804F066
:10144000A1FA281CFFF76AFF01E0FFF701FB37BD97
:10145000542B00209C2A0020DC050000F7B5494BE6
:101460000190000C984208D0474A1388002B01D104
:10147000108002E0834200D083E001AB5B78022B56
:1014800055D004D8002B11D0012B2ED079E0202B81
:101490006BD0242B66D0032B73D13C4D41232B7092
:1014A00001F0C0F90138C0B2394C3AE0394B0120A3
:1014B0001B78002B1FD1354D2B782E1C412B09D1C9
:1014C000334C277801F0AEF90138874202DA2078F0
:1014D00001301CE03078422853D12F4B198A023159
:1014E00089B21982FFF7C8FB4BE02A4B1B78002B0F
:1014F00004D001204042FFF73DFC42E0234D287814
:10150000412806D1224C207800283AD00138C0B2B8
:1015100007E0422835D1204B198A322931D90239C6
:10152000DEE7207001F060F928782178DAE7194CBD
:101530002378002B04D00120FFF70CFA00231FE0D2
:10154000124B1A78412A0BD142221A70124B1021E9
:101550005A5E002A01D1AF221A82198A4220C1E7BD
:1015600041221A70FFF7D8FB0BE00A4C01202378C8
:10157000002B02D0FFF7D2FE03E0FFF7AFF9012303
:101580002370F7BDFFFF00004A2B0020132A002024
:10159000142A0020982A0020FC29002010B5124CA3
:1015A0000021201C0522FEF703FE201C00F060FA3B
:1015B000002803D00D490E4AFFF714FC6378802BF6
:1015C00011D10C4BA022D205D4580B492140D15047
:1015D000D458C02189022143D150084B5B88DA07D7
:1015E00001D5FFF79BFE10BDA42A00200F040000C8
:1015F000DBB0020014070000FFFFFCFF682A002098
:1016000008B50120FFF732FB002803D00549064A40
:10161000FFF7E8FBBFF34F8F044A054BDA60BFF3D7
:101620004F8FFEE721050000DBB002000400FA0541
:1016300000ED00E008B5002801D0FFF7E1FF012030
:10164000FFF76CFE08BD000037B5041C4078103869
:101650000D284DD804F0B6F917074C4C4C364C2BDE
:101660004C4C4C324C436D460635A11C0222281CC2
:1016700007F0E6FC2B881F4A5904490C1BB2518025
:10168000002B35DA10E01B4DA11C281C022208306B
:1016900007F0D6FC281C211D0A30022207F0D0FCDE
:1016A000281C1E2100F0ECFEFFF73CFD20E0E27854
:1016B000A37812021A430F4B1A82F5E70120FFF7B5
:1016C0002DFE15E00C4B1B885A0611D500F0A6FA2A
:1016D000033843425841C0B200F0B6FA08E0A01CFB
:1016E00000F0BCFC002803D00449054AFFF77AFB50
:1016F00037BDC046682A002090FC03008A05000020
:10170000DBB0020008B5FFF7B3FA002803D00249A6
:10171000024AFFF767FB08BD4A060000DBB0020083
:10172000784BF7B500221A8080238022DB05D20097
:101730009958002900D09950734C1B59022B06D19F
:1017400000F0A6FC80230022DB051A5101E000F026
:1017500095FC6E4B05210093002006226C4B03F094
:1017600037FAAA21002800D0BBE06A4F0121381CBB
:10177000694A03F0A7FA002803D06849684AFFF7CE
:1017800031FB684E0121301C674A03F09BFA0028A8
:1017900001D06649F2E76648FFF784F908206549F9
:1017A0005022654B02F0B6FB002801D06349E5E703
:1017B000634802F0E7FBC821C9000028DED1FFF72B
:1017C0004DFA002801D05F49D8E70320FFF74CFA13
:1017D000002801D05C49D1E73420FFF743FA002804
:1017E00001D05A49CAE75A48FEF7B0FE0820011C4A
:1017F000584A03F015FBAF21002872D101F076FBA7
:10180000B621002811D1544C00213022201CFEF7B3
:10181000CFFC524D0021281C1422FEF7C9FC201CCD
:1018200001F07AFB002802D0BB214900A6E723780B
:10183000062B31D0E28806232370013A484B92B23E
:101840009A4202D983221201E280A288013A92B21E
:101850009A4201D9434BA3801022A35E013301D1E8
:1018600000232382A37CFF2B14D10723A374FA2324
:10187000DB00A3823C4BE3829623DB0023833B4BBC
:101880006383FA239B00A383E1239B00E383C823A4
:101890009B002384FFF746FC354B211C2B60354B06
:1018A00019206B6000F0B2FF334B00251D70334BE5
:1018B0004122E188281C1A7001F0FAF91E21201C2F
:1018C00000F0DEFD042000F071FBFEF7C1FF802177
:1018D0002A1C3868890103F01DFA021EAA4202D0B0
:1018E000A32189004AE73068254903F013FA00284C
:1018F00001D0244942E700F017F903F059FBFFF744
:1019000001FFFAE74A2B00201C050000E50C02004D
:1019100020270020AC2A0020290E0200AD02000082
:10192000DBB00200B42A0020990C0200B2020000D1
:1019300094240020182A0020FD0C02003C06000020
:10194000110D0200F4050000F9050000FC0500007F
:1019500068240020B82A0020682A0020FC290020E2
:10196000FDFF0000F41F0000140500004C040000FF
:10197000D044583B9A99193F142A0020132A00207A
:101980004E6240008F02000007B501AB187059701D
:101990003A20191C0222012301F0B6F80EBD13B53E
:1019A0000C1C694607310870012200233A2001F01F
:1019B000ABF80122211C131C3B2001F0A5F813BD3C
:1019C00037B56D46002307352B2040212B70FFF7DC
:1019D000DBFF6424013C2B20291CE4B2FFF7DFFF6E
:1019E000002C02D02B785A06F4D4631E9C41E0B23E
:1019F0003EBD08B52A200021FFF7C6FF08BD37B558
:101A000001F04AF8FFF7DCFFFFF7F3FF482115204C
:101A1000FFF7BAFF04211720FFF7B6FFFF212920A7
:101A2000FFF7B2FF04212B20FFF7AEFF08212C2087
:101A3000FFF7AAFF84212D20FFF7A6FF6C46842123
:101A40002E200734FFF7A0FF99212A20FFF79CFFE3
:101A5000211C0D20FFF7A3FF0025211C0C20257061
:101A6000FFF79DFF0B20211C2570FFF798FF37BD66
:101A700038B5411C041C0C20FFF791FF6378042546
:101A80002B420BD0A11C1620FFF789FF6119032000
:101A9000FFF785FFE11C281CFFF781FF63787F2B90
:101AA00003D90B20211CFFF77AFF002038BD23DF6C
:101AB000704727DF704728DF7047000000000000F4
:101AC000154908B54A68154B002A1FD000224A6004
:101AD000A1210120C90059585860A020C0001A5007
:101AE0009620C0004843FF2103F076FF03235843AC
:101AF00006F02AFC074B064A05F0C4FA04F090F8F9
:101B0000074B80B21B68002B00D0984708BDC04629
:101B10009A9999999999D93FFC70004000700040BA
:101B20005C2B0020C046C04608B5134B00225A600B
:101B30000720FFF7BEFF002803D06B210F4AFFF7F5
:101B400051F907200321FFF7B6FF002803D06E21CB
:101B50000A4AFFF747F90720FFF7A9FF002803D03B
:101B60007121064AFFF73EF9054BA0210122C90069
:101B70005A501A6008BDC046FC7000404BB10200CC
:101B800000700040F7B5041C081C01920D1C04F005
:101B9000A9FE1C4904F006FA071C04F027F80F23DD
:101BA000061C1E40301C04F09DFE011C381C04F075
:101BB00003FD154904F0D4FB04F018F8134AC0B231
:101BC000012395420CD8124A0223954208D8114AA3
:101BD0000323954204D8104A0023AA425B410433F0
:101BE00062780F218A4307210B40164370221B01A4
:101BF00096431E437F22019B164020706670201C76
:101C00006360FEBD00007A4400007F43DC1E0000DC
:101C1000B01D0000841C0000901A0000094B10B594
:101C20001B8800205A060CD5A021A222D200C9058B
:101C30008C5888580123C00A1840620A9840134003
:101C4000184310BD90FC0300084B1B885A060CD5A6
:101C5000074901220978A023DB058A40002801D02A
:101C6000044901E0A121C9005A50704790FC0300CB
:101C7000602B00200C050000074B1A60074BC122A7
:101C80001870074B92001970064B012199500649B4
:101C9000064A99507047C0465C2B0020582B002004
:101CA000602B0020007000400808000004050000C0
:101CB00014220D4B504330B51B68C058002301223D
:101CC0009A4010420BD0A022D20599008918E02238
:101CD000D2008D58054C2C408C508C588C500133C0
:101CE000202BECD130BDC046682B0020FFFFFCFF4D
:101CF000F0B5002301229A40114217D00468144223
:101D000003D122430260802502E094430460C02591
:101D1000A022D2059C00A418E022D200A758054EAC
:101D2000AD023E40A650A6583543A5500133202BA6
:101D3000E0D1F0BDFFFFFCFFF7B5A223A022DB003E
:101D4000D205D5582149BE22002352008B501F1CBA
:101D50001F4B1B78BB4237D91E491F4B0122096814
:101D6000BA401B6811422CD014247C431C19E36830
:101D700026686B40221C0C329E43101C311C0192C1
:101D8000FFF7B6FFA223A022DB00D205D3586B4099
:101D90000BD01D43E36822686B409A430198111CE5
:101DA0000092FFF7A5FF009B1E43A1686068A9434E
:101DB00028400B1C03431E4203D0304031402369AE
:101DC00098477B1CDFB2C3E7F7BDC0460060004008
:101DD000612B0020642B0020682B002038B50029DF
:101DE00026D003240C4023D1134B14221960134B2B
:101DF00042431870124B081C1C70124B211C1C60B3
:101E0000FEF7D6F9104A0121C22349429B00D15066
:101E10000E4BC021402249005A50C12189005D5813
:101E20000B482840C0252D04284358501A6000E074
:101E30000724201C38BDC046682B0020622B0020E0
:101E4000612B0020642B00200060004000E100E0D6
:101E5000FFFF00FFF8B5061C11480568002D1AD0D9
:101E6000002B1AD00F48104F00783C78844604208D
:101E7000A44513D9142060432D18081C1043286072
:101E80002B616960AA60631C201C34703B70FFF7F3
:101E90000FFF002002E0082000E00720F8BDC04648
:101EA000682B0020622B0020612B0020244BF7B50B
:101EB0001A68002A41D0234B1978072381423DD963
:101EC0002149BE2300245B00CC50A223A024E405BA
:101ED000DB00E3581D4C01932368002B04D18027BD
:101EE000C1263F06B6008F51012181400B4323607C
:101EF00014235843101800230668C36001229A4037
:101F0000164215D00199C024114203D1C56880241E
:101F10002A43C260A027FF059900E022C919D20018
:101F20008D580B4FA4022F408F508F583C438C503C
:101F30000133202BE2D1002300E00823181CFEBD52
:101F4000682B0020612B002000600040642B0020E3
:101F5000FFFFFCFF014B18607047C0466C2B002050
:101F6000A223A022DB00D205D2580D4B10B51B686E
:101F7000DA400C4BD10708D418780130C0B2187081
:101F8000283843425841400009E0197800220239BC
:101F90002520C9B2141C88425441E0B21A7010BD09
:101FA0006C2B0020702B002051DF704708B5054BCB
:101FB0003021187007F038F8034B1860434258413D
:101FC000800008BD712B0020742B002070B50A4BD7
:101FD0000A4C1978207803F043FD3022CDB25543E6
:101FE000074E002133685819FEF7E2F8237830686D
:101FF00001334019237070BD712B0020722B00201B
:10200000742B002008B5074B1878074B013019785E
:1020100003F086FD3020C9B24843044B1B681818F2
:1020200008BDC046722B0020712B0020742B0020AD
:1020300008B5074B1978074B18784018023803F099
:102040006FFD3020C9B24843034B1B68181808BD08
:10205000712B0020722B0020742B002007B5002369
:10206000011C042201A8019306F0EAFF024801A91D
:102070000422FFF799FF0EBD90FC030008B5C422AF
:10208000024800215200FEF793F808BDB02400205A
:1020900000487047B024002010B50F4C23886060C2
:1020A000201C013361800830111C7F22238007F03F
:1020B000B6F8231C873300221A70084B69461A6849
:1020C000201C80238830521A5B009A4200D91A1CC7
:1020D00006F0B6FF10BDC046B0240020000002008C
:1020E00023DF704724DF704728DF704742DF7047E7
:1020F00044DF704708B5074B01225A600A20DA60B6
:10210000FFF7F0FF044A00231370044A1370044AD7
:10211000137008BD00A00040802B0020792B002008
:10212000782B0020194B012270B51A70184B00242F
:102130001D68A023A222DB05D2009A581E1CEA408B
:10214000D30716D50134E4B2152C12D06423C0464F
:10215000C046C046C046C046C046C046C046C0464F
:10216000C046C046C046C046C046013B002BEED12B
:10217000DFE7FFF7BFFF0020142C05D90123AB4098
:102180001D1C044B0820F55070BDC046792B002063
:102190007C2B00200C050000F8B5174B051CC2185D
:1021A000B0230720DB009A4225D8144E3378002B49
:1021B0001DD1134CA823DB00E550124B6D00E550F8
:1021C000114B6D42ED18A923DB00E5500F4B0027A2
:1021D0001F708022C1230125D2029B0035700A2086
:1021E000E250FFF77DFFE560381C256003E0FFF754
:1021F00099FF0028DDD0F8BD45FDFFFF802B0020B2
:1022000000A0004044050000204E0000782B002074
:1022100008B5E022274B520018608118A023DB0587
:1022200089000122CA50244982405A502349244B34
:10223000244AD150C046C046C046224B0122DA6033
:10224000214A000210431E4A9850C046C046C0466C
:1022500004201E491E4AFFF74BFF002803D07C21B3
:102260001C4AFEF7BFFD05201B49194AFFF740FF36
:10227000002803D08221174AFEF7B4FD3020FFF773
:1022800035FF002803D08821124AFEF7ABFD134B1F
:10229000134900225A50A121C9005A50A2220421F8
:1022A000D20099500122DA600A200321FFF71CFFB7
:1022B00008BDC0467C2B00200C050000031F020057
:1022C0001C050000006000400300030040A1004026
:1022D0000C60004062B1020044A1004000A0004038
:1022E000040500000E4A08B5D16C0E4B002906D03B
:1022F000C12189005958480301D50021D1640A4AF7
:102300001278002A02D0FFF7F5FE07E007490A78A5
:10231000501C0870312AF6D80122DA6008BDC04688
:10232000FCA0004000A00040792B0020782B00206A
:10233000F7B506F03DF83F4B3D4A041C0D1C07F075
:1023400093FB3D4A3D4B061C0F1C201C291C07F02B
:102350008BFB3B4A3B4B00900191301C391C05F034
:10236000B9F9394A394B061C0F1C0098019905F040
:10237000B1F9021C0B1C301C391C04F05FFB344A01
:10238000344B061C0F1C201C291C07F06DFB324A25
:10239000324B05F09FF9021C0B1C301C391C05F058
:1023A0002BFC2F4A2F4B061C0F1C201C291C07F04E
:1023B0005BFB2D4A2D4B05F08DF9021C0B1C301CCC
:1023C000391C04F03BFB2A4A2A4B061C0F1C201C1C
:1023D000291C05F07FF9021C0B1C301C391C05F070
:1023E0000BFC254A254B04F029FB06F033F8041CAE
:1023F00000F0C4F904F076FA011C201C03F0C2FBC3
:10240000002802D000F0BAF910E000F0BDF904F0A5
:1024100069FA011C201C03F0A1FB002802D000F087
:10242000B3F903E0201C03F0E1FB80B2FEBDC0461F
:1024300000000000000014400000000000001040F8
:10244000B93520605DAA18BFF30EBA8DE72A863F22
:102450000000000000000840D68F6E6D248DDD3F27
:1024600000000000000000408EFCB94D93ED2140BB
:1024700076F0515764E15540EDA22A4AE959984057
:10248000F7B5194B041C00890191184D184F194ECE
:1024900098420FD004F026FA174903F083FD286014
:1024A000608904F01FFA144903F07CFD00233860B2
:1024B000336017E0A08804F015FA104903F072FDAC
:1024C0000F4903F04DFF041C019804F00BFA0A4970
:1024D00003F068FD011C201C03F042FF094B306033
:1024E0002B603B60F7BDC046FFFF00008C2B002037
:1024F000882B0020842B002000007A440000C84272
:10250000C3F51C4100FF7F47F0B589B0C78B061C9F
:102510000591049200F032F9874270D200F034F94C
:10252000874205D2072055216D4AFEF75BFC60E02B
:10253000381C05F009FF574B554A0290039107F0EC
:1025400093FA554A554B041C0D1C0298039907F049
:102550008BFA534A534B06900791201C291C05F017
:10256000B9F8514A514B041C0D1C0698079905F007
:10257000B1F8021C0B1C201C291C04F05FFA4C4A09
:102580004C4B041C0D1C0298039907F06DFA4A4A43
:102590004A4B05F09FF8021C0B1C201C291C05F05F
:1025A0002BFB474A474B041C0D1C0298039907F06C
:1025B0005BFA454A454B05F08DF8021C0B1C201CAC
:1025C000291C04F03BFA041C381C0D1C05F07EFE8F
:1025D0003F4A404B05F07EF8021C0B1C201C291CB6
:1025E00005F00AFB3C4A3D4B04F028FA05F032FFA7
:1025F000041C201C002103F0B1FA002800D00024A4
:10260000384B39491F68381C03F0A2FA00280ED154
:102610007568391C281C03F0A3FE344B196803F0BD
:10262000CBFF291C03F0BEFC0499086003E0304B8B
:10263000049A1B681360049B201C196803F046FB76
:10264000716803F08DFE04F02DF90599338A0A8A2A
:1026500080B27080934200D2013B9B1A00229BB251
:1026600090420BD0934209D000B2584304F03AF99B
:10267000204903F097FC03F0B9FA82B205990020D3
:102680000B89D218328109B0F0BDC046C046C046A1
:102690000000000000001440000000000000104096
:1026A000A08136F5E9D075BD882D403D3CFC3C3E0F
:1026B00000000000000008401366DD7CAEB3ED3E74
:1026C0000000000000000040A2B75A5C6F368D3F4A
:1026D00087A77D35A5B61B402E3B78B1DA1D954006
:1026E00079B102008C2B002000FF7F47882B00204F
:1026F000842B0020D00FC943014B18887047C04677
:10270000942B002038B5184B1B689A7C0732520076
:102710009A189488A04205D39A8A041C904200D942
:10272000141CA4B2114D2A88A2421BD0A11A02295E
:1027300002DC121B022A15DD188AFA23201880B247
:10274000DB00984204D80A4B984202D8094800E0BE
:10275000181CFFF721FD002803D08321064AFEF74D
:1027600041FB2C80288838BD902B0020942B002022
:10277000BA020000BB0200008EB10200014B1B68D0
:10278000988A7047902B0020034B1B689A7C073275
:1027900052009B1898887047902B002070B50278E3
:1027A000011C00200A2A18D80C4B1C68031C580076
:1027B00008184088FA25ED00A84207D0258A084E5F
:1027C000AD194019074D80B2A84205D80133D8B2DF
:1027D0009042ECD3012000E0002070BD902B00203F
:1027E00045FDFFFF1505000008B5074B1B689A7CE7
:1027F000904201D3501EC0B2083040001B18988888
:10280000FFF780FF08BDC046902B002008B5044BA1
:102810001960FFF7FDFC0020FFF7E6FF08BDC0468A
:10282000902B0020014B1B68987C7047902B002058
:10283000F8B50021041C03F08BF9174D002802D0D5
:102840002B68988A24E0201C144903F09BF9002887
:1028500006D02B689A7C073252009B18988817E0A4
:102860002D68AE8A301C04F03DF8AB7C071C0733A2
:102870005B00ED18A888301A04F034F8211C03F02E
:102880006FFD011C381C03F097FE03F0AFF980B216
:10289000FFF738FFF8BDC046902B0020CDCCC742D3
:1028A000F7B5051C161C1C1C002809D0486869686F
:1028B00003F00CFAFC21890503F052FD071C00E02F
:1028C0004F688021381CC90503F048F9002859D108
:1028D000422C02D0432C0BD054E01023F05E04F0C5
:1028E00001F8391C03F05EFB089903F065FE45E032
:1028F000706805F05DFD041C0D1C381CB16803F008
:10290000E5F905F055FD214B1F4A07F0ADF8224BC4
:10291000009001911B68988803F0E4FF1F4903F0C1
:1029200041FB1F4903F01CFD009A019B071C291C59
:10293000201C04F0CFFE164A164B04F0CBFE05F027
:1029400089FD3168041C381C03F00AFD011C201CA1
:1029500003F0BCF9F168041C381C03F001FD011CF4
:10296000201C03F0B3F9089903F026FE0021041C93
:1029700003F0F4F8002800D00024201CFFF7D8FC56
:10298000FFF7C0FEF7BDC046000000000000004099
:10299000000000000000E03F902B00200000C84233
:1029A000C3F51C41C046C04682B00190C046C04637
:1029B000C046C046C046C046C046C046C046C046E7
:1029C000C046C046C046C046019B013B0193002B58
:1029D000ECD102B0704742DF704743DF704744DFFD
:1029E00070470000F7B5A023274EDB00F158002206
:1029F0000091264DF250A024254AE405E8236759AA
:102A0000DB006251E15804200191E250A1238022B1
:102A1000DB005202E25080221202E250FFF7C4FFB4
:102A2000A223DB00E258D10304D5E2580123D20BE4
:102A30001A4217D11324013C002C15D0154BA025A8
:102A40008026ED053602EE500420FFF7ADFFA123EE
:102A5000DB00EE500420FFF7A7FFA223DB00EB58BA
:102A6000DA03E8D5012000E0201C0849A023DB059B
:102A70005F50E8220199D20099500099024AA023A0
:102A8000DB00D150FEBDC046004000403C070000C6
:102A90000D0600000C050000144A1549A023DB05B3
:102AA00010B55A50134CE821C9005A50231CFC336E
:102AB0000022DA601A62A1230F22DB00E2500E4BE3
:102AC0001022E2500D4BCC225204E2500C490D4A28
:102AD0000620FFF784FF4020FFF77FFFA023052299
:102AE000DB00E250FFF77EFF10BDC0460C06000081
:102AF0003C070000004000400C05000024050000D9
:102B0000384100401C400040F7B5071C0091161CDE
:102B1000019301D100209CE0FFF764FF0028F9D069
:102B20004C4CB123DB007A08E25001234A4D1F428E
:102B30004CD0062049499E4201D1494A00E0494A09
:102B4000FFF74DFF4020FFF746FF0023EB60464FA5
:102B500001232360EB68002B06D13F4B9B6A002BBF
:102B600002D1013F002FF5D10023EB609F4248D0F6
:102B7000394B9B6A002B44D1364AA323DB00D35840
:102B8000009A00981370731E0130DEB20190012E7E
:102B900005D13249324A0620FFF721FF01E0002E1D
:102BA00007D01420FFF700FF01232362019B00934D
:102BB000D0E72D4BAA68002A02D1013B002BF9D1A6
:102BC0000023AB604020FFF708FF39E0009F009A28
:102BD0003978264F0132E151A360234B296A00293D
:102BE00007D11D49896A002903D1013B002BF5D18A
:102BF00007E0002B05D0AF6A16491748BC46002FE6
:102C000010D00026AE621A4FA025ED0066510520B7
:102C1000E651FFF7C9FE0123E35105236351FFF796
:102C20003BFF77E7013E6746F6B20762002E04D00D
:102C300010780E4F0132C851D0E7019F002F01D10B
:102C4000012006E0012386604B61AB68002BFCD0BD
:102C5000F6E7FEBD00400040FC4000403841004027
:102C6000144000401C400040204E00001C050000A5
:102C7000FC0F000042DF704744DF704708B5084B87
:102C8000188003F02FFE074903F08CF9064903F082
:102C900089F9011C03F01AF8044B186008BDC046FE
:102CA0009C2B002000007A441F85EB3D982B0020D0
:102CB00010B5041C081CFFF7E1FFE0235B00E218DD
:102CC000A02392000021DB05D150184B24021C43A5
:102CD000174AA323DB00D450C046C046C046154B5C
:102CE0000022DA6003201449144AFFF7C5FF0028C8
:102CF00003D04A21124AFEF775F80820FFF7BAFF01
:102D0000002803D04D210E4AFEF76CF80D4B0E49FA
:102D100001225A50A1210020C90058500B4980209F
:102D20008000DA6008601A6010BDC0460100030030
:102D300000600040FC6000400861004008900040D6
:102D4000A8B10200009000400405000000E100E08E
:102D50003B4BF7B501221A64A822D2009E58041CEE
:102D600046614A690B8AB01A00935AD025880F88A9
:102D7000BD4202D26B1EDF1B00E0EF1B03F00EFE14
:102D8000304903F00FF9BFB20190381C03F0AAFDDF
:102D9000E821890503F0E4FA011C019803F002F927
:102DA000071C6060301C03F0F9FD274B196803F025
:102DB000F9F8061C02F01AFF244BE060188803F0B3
:102DC00091FD011C381C03F0EDF8011CFE2080056C
:102DD00003F0E8F81E4903F0E5F88A21C90503F07D
:102DE000BFFA02F003FF009A87B2BB182382301C9F
:102DF00005F0DEFA114B104A06F0CEFD05F02AFB75
:102E0000061C381C03F0CAFD011C301C03F0A8FA94
:102E100005F0CEFA06F060FD02F002FF2D1A2583C0
:102E200007E0CB68009AE3600B8B228223830023A8
:102E300063600020FEBDC046000000000000F03FBF
:102E40000090004064218B41982B00209C2B002097
:102E500000007A44C046C04607B5012301A990206E
:102E600002220B704B70FFF74FFE07BD37B50423EE
:102E70006C46E370012203340025211C131C9020B2
:102E8000FFF742FE211C2570012201AC2B1C902073
:102E9000FFF73AFE022201239120211C2570657064
:102EA000FFF732FE237860781A0100095BB2104305
:102EB000AB4206DA03F016FD8B21C90503F07CFB5B
:102EC00001E003F00FFDF621890503F049FA3EBD4C
:102ED00007B5202201A901234A70902002220B701D
:102EE000FFF712FEFFF7C2FF07BD704707B502F0FC
:102EF000B5FB00280AD130236A4693800123D38092
:102F0000034B68460349009302F012FC0EBDC04615
:102F1000EB2E0200A02B002008B50349302200232D
:102F200002F0C4FC08BDC046A02B002038B5084CF8
:102F3000051C3021201C02F0F3FC031E05D1201CCF
:102F4000291C302202F070FC031C181C38BDC0463E
:102F5000A02B002008B5437800781B02184303F02B
:102F6000C1FC024903F01EF808BDC04600401C46E3
:102F700008B5437800781B02184303F0B3FC0249FC
:102F800003F010F808BDC04600007A4408B5437845
:102F900000781B02184303F0A5FC011C034803F052
:102FA0000BFB024902F0FEFF08BDC04600FC7F4655
:102FB00008B5437800781B021843044B584000B210
:102FC00003F090FC024902F0EDFF08BD0080FFFF16
:102FD00000007A4408B5437800781B021843054B7B
:102FE000584000B203F07EFCE021890503F0B8F9F7
:102FF00008BDC0460080FFFFC2DF7047C4DF7047D6
:10300000C7DF7047C8DF7047CCDF7047CDDF704740
:10301000D1DF7047D3DF704708B5021C08210120BB
:10302000FFF7EEFF054B984206D0054A83185A1E5B
:1030300093415B42184000E0002008BD22400000A0
:10304000E1BFFFFFF0B50A4B49001D785918002376
:10305000DCB2AC420BD2944209D2467807785C00CD
:1030600036020C193E43668001330230F0E7F0BDB2
:10307000CE2B002070B58478051C64090BD10F4E4F
:10308000211C1622301CFDF793F82B79681D337034
:10309000211C03220EE0042203300321144209D034
:1030A00007210322FFF7CEFF054B04481B689B6AEC
:1030B000984701E0FFF7C6FF70BDC046CE2B002049
:1030C000C02B00201FB5522402AA1470FF24031C39
:1030D0005470000A11249470D1700C0AC0B2090C0B
:1030E000517193717021C3090140DB01194300073D
:1030F000030F081C1843D071082101201471FFF739
:103100007FFF04B010BD000037B5C378041C502BFE
:1031100031D101792F4B490911D12F4A012010706B
:1031200062791A70482A02D0592A20D050E02B4DDB
:103130000822281CFDF73CF8A3792B7048E00422F4
:10314000114211D0244A117800290DD01B7800219A
:103150001170482B09D1224A204B1268411D596039
:1031600052691868904733E01B78592B30D1A01C66
:10317000FFF780FF2CE04F2B2AD14379462B22D03A
:10318000F02B06D0022B23D1154B05301B685B6A50
:103190001DE08379612B0AD0642B03D0602B17D1FB
:1031A0005C2305E00E4B1B68DB69984710E05B234E
:1031B0006A46211C13700831094B01911B68009865
:1031C0005B69984704E0064B05301B681B6A98470B
:1031D00037BDC046CC2B0020A92B0020AC2B0020F3
:1031E000C02B002008B52B4B2B4918600020FFF79F
:1031F0000BFF002804D0D821FF31284AFDF7F2FD4B
:10320000002201201021131CFFF7F6FE002804D035
:10321000DE21FF31214AFDF7E5FD80235B05596E74
:10322000012089B20B22A523FFF7F4FE002804D069
:10323000E421FF31194AFDF7D5FD01203921FFF7BF
:10324000E5FE002804D0F3214900144AFDF7CAFD29
:1032500001201349FFF7DCFE002804D0EA21FF31EA
:103260000E4AFDF7BFFD0F4A10231370FF21002304
:1032700053709170D170137153719371D3710A4A65
:103280001120107053709370D1701371537193713A
:10329000D37108BDC02B0020BDB10200C5B1020032
:1032A000F61F0000B52B0020C42B002008B501201C
:1032B000FFF7A4FE002803D00249034AFDF792FD60
:1032C00008BDC04603020000C5B1020037B5494B36
:1032D000041C1D78F2210135EDB21D70281C02F08E
:1032E000BFFBC9B200290FD101200821424AFFF7D4
:1032F00087FE424B984200D17AE0414B984277D00A
:10330000002875D03F4970E0281C792102F0A8FB05
:10331000C9B200290ED1012008213B4AFFF770FEF7
:10332000364B984264D0364B984261D000285FD02B
:1033300036495AE0281C3D2102F092FBC9B200290F
:1033400004D1A06AE16AFFF7BDFE51E06A071FD110
:103350006A4624231370E38B206A53701B0A937010
:10336000A38BD370A27E1B0A403AD2B292011343C0
:103370006A461371636953711B0A937102F036FC3C
:103380006B46D87108216A460120FFF739FE2FE00D
:10339000281C052102F064FBC9B2002914D11C4885
:1033A000618803888AB2D3189BB203801948120A35
:1033B00003711B0A457043718171C271FFF72CFEC6
:1033C000002815D0144910E023891448228A217B53
:1033D00002718371120A1B0A457081704271C371B8
:1033E000FFF71AFE002803D00D490E4AFDF7FAFC3C
:1033F00037BDC046B42B0020602F002022400000C3
:103400001F40000016020000582F00201A02000082
:10341000E42B0020B52B002029020000C42B002043
:1034200031020000C5B1020007B5F0236A461370EF
:10343000802350709370094A684613780133DBB2D9
:1034400013706A46D370012311719371090A002326
:103450005171D371FFF7E0FD0EBDC046A82B0020CF
:1034600073B502236D462B700B786870AB704B7888
:10347000EB708B782B71CB786B710B79AB714B79CF
:10348000EB710425802A19D1013DEDB2114E002DBA
:103490000ED0012008216A46FFF7B4FD041EB44295
:1034A00002D00D4B98420DD1052002F06BFAEBE7EC
:1034B000B4420ED0084B9C420BD003E06846FFF7A5
:1034C000ABFD041C002C04D0201C0449044AFDF769
:1034D00089FC73BD224000001F40000083020000F1
:1034E000C5B1020073B506AC0025645F6E460325C6
:1034F0003570051C0F2800D90F25684603718471AB
:103500001B0A240A45708170C2704371C471FFF7B1
:1035100083FD002803D00249024AFDF763FC73BD16
:10352000AB020000C5B10200C2DF7047C4DF7047C4
:10353000C7DF7047CDDF7047D1DF7047D3DF7047FB
:10354000002208B503201021131CFFF7EDFF00280F
:1035500003D03D21134AFDF745FC80235B05596EDE
:10356000032089B27B220123FFF7E8FF002803D064
:1035700043210C4AFDF736FC03203921FFF7DAFF1F
:10358000002803D04621074AFDF72CFC03200649FA
:10359000FFF7D2FF002803D04921024AFDF722FCA1
:1035A00008BDC046E2B10200B61F000008B5032006
:1035B000FFF7BCFF002803D05421024AFDF712FC9C
:1035C00008BDC046E2B10200F8B52B4B071C1D78C0
:1035D0000E1C2A4CAA0707D123787F21DA09D2438F
:1035E000D2010B4013432370281C822102F038FAC9
:1035F000C9B2002909D122787F239A4303231A43B1
:1036000063702270A17048231BE0281C412102F046
:1036100027FA22787F239A43C9B2131C00290CD1C0
:103620000222134323705D23637080235B055A6E6F
:10363000120CA2705B6E1B0E03E0FF2322706370FE
:10364000A3702771A6713F0A360A03200821221CA5
:10365000E3706771E671FFF76BFF094B984206D084
:10366000084A83185A1E93415B42184000E000202C
:10367000014B01351D70F8BDE62B0020A42400206D
:1036800022400000E1BFFFFFC2DF7047C4DF704788
:10369000C7DF7047CCDF7047CDDF7047D1DF7047A1
:1036A000D3DF704738B5244D244B254C196020706A
:1036B0000021281C0822FCF77BFDFF230020214964
:1036C0006B70AB70EB70FFF7E5FF002803D0A6210D
:1036D0001D4AFDF787FB002220781021131CFFF7FD
:1036E000D3FF002803D0AD21174AFDF77BFB8023D1
:1036F0005B05596E207889B210220523FFF7D0FFB1
:10370000002803D0B421104AFDF76CFB2078392142
:10371000FFF7C2FF002803D0B7210B4AFDF762FB79
:10372000802120788901FFF7B9FF002803D0BA2152
:10373000054AFDF757FB38BDEC2B0020E82B002095
:10374000E72B002007B202000FB2020008B5054BBC
:103750001878FFF79BFF002803D0C321024AFDF72A
:1037600041FB08BDE72B00200FB2020073B5082211
:10377000041C2449684605F063FC234E6B463078F0
:1037800008216A465C70FFF783FF002803D0DB2125
:103790001E4AFDF727FB1E4C822125780135EDB22C
:1037A0002570281C02F05CF9C9B200290ED13078CE
:1037B0000821184AFFF76CFF174B98421ED0174B91
:1037C00098421BD0E321002818D014E0281C412186
:1037D00002F046F9C9B2002913D130780821104A05
:1037E000FFF756FF0C4B984208D00C4B984205D07F
:1037F000002803D0E821054AFDF7F4FA23780133C5
:10380000237073BDFFB10200E72B00200FB202004E
:10381000F42B0020602F0020224000001F400000F9
:10382000582F002013B54379462B02D0492B10D0D6
:1038300029E0C37A472B26D1134B08211878134A65
:10384000FFF726FF00281ED09221114AFDF7CAFA81
:1038500019E00E4C827AA1780530914213D0237082
:1038600004238179E37001AB1A70A27082785970D9
:103870006170417812020A435A80064B01981B6816
:1038800098470023E37013BDE72B0020EC2B0020AA
:103890000FB20200E82B0020A0DF7047A2DF7047C4
:1038A000A6DF704762DF704770B54B88041C9370C9
:1038B0001B0AD37000680223034008D00B89002B39
:1038C00005D013711B0A53710620042300E0042065
:1038D0002468650715D5CC68002C12D01025260A5F
:1038E0002B4315182C706E70260C240EAE70EC70E5
:1038F0000C8B011DC9B251180C700630240A4C7093
:10390000C0B213700023537070BD73B50B88051CD3
:103910000C1C112B06D0502B09D0102B1ED18B88DC
:10392000803502E0012380355B422B8016E0031CCA
:103930007833CA881B888E1D9A420FD10021082235
:103940006846FCF735FCB37E6A461370211C2B6871
:1039500021310191002B01D00098984773BD0000E0
:10396000F0B5ADB00591031C0969012280335242C4
:1039700001601A80059A20AC92680490826002234C
:10398000DF48211C2370FFF78DFF002803D0422160
:10399000DC4AFDF727FA049ADB4B08A90120043220
:1039A00088700B80FFF778FF002804D0E821FF31F2
:1039B000D44AFDF717FA00211C22201CFCF7F8FB63
:1039C00023780826334320221343D04A102010AF17
:1039D0000221051C3A80012215438C46B9700BA9BF
:1039E0000D70051C15434D708D780626B54366464F
:1039F00035430826B54385432A43049D8A702370C6
:103A000017AA00236360E36023616361A3615160CF
:103A100013810421538113612B1C9181A888211CDF
:103A200078331797FFF73AFF002804D0EC21FF31D5
:103A3000B44AFDF7D7F920AC00211C22201CFCF76A
:103A4000B7FB237802273B432370B14B6D462E21F1
:103A50000026AB8501220AAD69440A70281C311C7E
:103A600003226660E66026616661A661FCF7A0FB42
:103A7000059906220B7F2B704B7F311C6B70AB7846
:103A800093431F43E7231F4001229743AF7017AFB3
:103A90001422381CFCF78CFB059B7E819A68049EDF
:103AA00010AB110A1A705970110C120E9970DA705D
:103AB0000BA904223B61331C17913A81BA81B0886B
:103AC000211C3A1C50337D60FFF7E8FE002804D02B
:103AD000F021FF318B4AFDF785F98E4B002103223F
:103AE00006A810270A93FCF763FB012369463B43B2
:103AF0000B7601233B434B768B7E062202269343B3
:103B0000334310AE8B761C220021301CFCF750FB97
:103B10003378281C3B433370756005F079FB26220F
:103B200001236A4407AC80B206A913707A4B308136
:103B300070817161B1616D46201C00210322AB844C
:103B4000FCF736FB059D0621EB7F022223702B1C20
:103B50000133DB7F01256370A3788B431343082275
:103B60009343BB432B430BAD17AF00211422281CFA
:103B7000A370FCF71DFB00212222381CFCF718FB68
:103B8000049809A96C6020AC0B913A1C211C0830E8
:103B9000FFF78AFE00236B812223049AAB81049BEA
:103BA0002881311C908858332A1C2F61FFF776FE3C
:103BB000002804D0F421FF31524AFDF713F9002107
:103BC0001C22201CFCF7F4FA2378022633432370CE
:103BD000422301216B441970504B00250BAF10AAF2
:103BE0001380291C0322381C6560E560256165612E
:103BF000A561FCF7DDFA059B06229B19DB7F291CDA
:103C00003B70059B0333DB7F7B70BB7893431E4384
:103C1000E7231E4001239E43BE7017AE1422301CC2
:103C2000FCF7C6FA7581059D01226D6810A9356102
:103C3000049D17912B1C3281B281A888211C321C53
:103C400060337760FFF72AFE002804D0F821FF31A7
:103C50002C4AFDF7C7F8059E3378002B4CD020ADD9
:103C600000211C22281CFCF7A3FA2B7808210B4307
:103C7000202213432B704222294B002401260BAF34
:103C80006A4410A916700B800322211C381C6C603A
:103C9000EC602C616C61AC61FCF78AFA10231A1C91
:103CA00032433A701A1C32437A70BA7806218A433A
:103CB00002210A4308218A439A43131CB34317AED7
:103CC000211C1422301CBB70FCF772FA0423B38150
:103CD000049B10AA17929888291C6833321C7760BD
:103CE000348174813461FFF7D9FDA04204D0FE21F4
:103CF000FF31044AFDF776F800202DB0F0BDC04634
:103D000026B2020036B202001818000005E0FFFFDC
:103D1000652A000043504D00632A00005D2A000020
:103D2000662A0000F0B5021C803291B000921A4B56
:103D30001288071C0C1C08209A422AD007AE0021CA
:103D40002222301CFCF734FA381C211C321C0830AB
:103D5000FFF7AAFD03AC6D46688101900021102297
:103D6000201C5837FCF724FA3B88009A2380012353
:103D70000A35A37010880023211CA380A560E6608B
:103D8000FFF78EFD002804D12B88019A934200D0C2
:103D90000C2011B0F0BDC046FFFF0000F0B5031CC1
:103DA000803389B001931988144B071C082099426D
:103DB00022D003AE04AC32706B46C2405A736D46DB
:103DC00004230021201C102278376B81FCF7F0F9C6
:103DD0003B880A3523800223A3700023A380019B24
:103DE000211C1888A560E660FFF75AFD002803D162
:103DF0002B88042B00D00C2009B0F0BDFFFF000081
:103E000023DF70474EDF704710DF704760DF704779
:103E1000C1DF704708B5081C111CFCF71DFB08BD6D
:103E2000F0B5354B87B01B78002B63D0334D344E43
:103E30002968344F4B424B413168DBB203934B420C
:103E40004B413968DBB201934B424B41DBB20293E9
:103E5000039B002B11D105A8FFF7D4FF05280AD03A
:103E6000002804D06921284AFCF7BCFF05E005982A
:103E70002968884701E0012303930199002917D19C
:103E8000224B05A91B880B80214B1C68201CFFF7C7
:103E9000BDFF05280AD0002804D080211A4AFCF76B
:103EA000A1FF05E0201C3368984701E00121019142
:103EB000029B002B02D00121029112E0144B1C68DE
:103EC000611CA21C201CFFF7A3FF0528F3D00028CB
:103ED00004D098210C4AFCF785FF02E0201C3B68C7
:103EE000984703990029B3D0019B002BB0D00299C9
:103EF0000029ADD007B0F0BDF52B0020FC2B002031
:103F0000042C0020F82B00204CB20200F62B0020DD
:103F1000002C002038B5041C0720002913D08D0781
:103F200011D1094801600949201C0A80084A094941
:103F30001360FFF769FF002805D1074B0122162007
:103F40001A70FFF75DFF38BD002C0020F62B002013
:103F5000082C0020153E0200F52B0020002803D07D
:103F6000024B1860002000E00E207047042C002057
:103F7000002803D0024B1860002000E00E2070479C
:103F8000F82B0020002803D0024B1860002000E02E
:103F90000E207047FC2B002008B5084B1B68002B37
:103FA00008D09847002807D099214900044AFCF717
:103FB00019FF01E0FFF734FF08BDC046082C0020C0
:103FC0004CB2020072DF704779DF70477DDF7047C7
:103FD00064DF7047F0B587B00C9F061C387800246A
:103FE0000391029200930190251C33889D4238DA98
:103FF0007268A900511805A8042205F021F8694645
:1040000005A813310022FFF7E3FF002832D16846EC
:10401000C37C02998B4220D1624262413B785200BC
:1040200059188A181F2A1ADC002C06D19A1C3A70DB
:1040300001330398009ADBB2D05400996C463A7869
:1040400013348A1805A8211CFFF7C2FF002811D1DC
:104050003A7823780124D3183B700135C5E70C204A
:1040600008E00020844205D03B78019A013B00998A
:104070009B1A8B5407B0F0BDF7B5089E171C00962D
:104080000222051C1C1CFFF7A5FF002806D1009684
:10409000281C391C1022231CFFF79CFFFEBD0000CA
:1040A000F0B500231370037887B0061C0D1C141C98
:1040B000002B03D1B378002B47D027E043780C20A6
:1040C0001D2B00DD53E16F4616371D23881C391C5C
:1040D0003B80FFF77BFF002800D048E13378022BBC
:1040E00003D13B8809221D2B07D97378002B02D0FE
:1040F00008221D2B01D93B880822DBB2591C2970EC
:104100006A70227802329B182370D3E723780C2040
:104110001B2B00DD2BE16F461637381CFFF754FFD1
:10412000002800D023E1237839885A1C227003220A
:10413000EA5423785A1C22701922EA542378EA1888
:1041400011700233090A51702370B288002A1ED000
:10415000B168002900D109E123780C20991C8A1844
:104160001F2A00DD03E15A1C2270B2880132EA5492
:1041700023785A1C22700122EA542078B288281829
:10418000B16804F05DFFB2882378D3182370F36818
:10419000002B12D01A7823780C201C2B00DDE6E0CF
:1041A000591C21700221E9542378591C21700A21DD
:1041B000E9542378591C2170EA54338A002B03D127
:1041C000338B002B16D00AE0301C009410300221F3
:1041D00006222B1CFFF750FF0028F1D0C7E0301C4F
:1041E00000941830032107222B1CFFF745FF0028FD
:1041F00000D0BCE0338C002B0AD0301C009420305F
:10420000142115222B1CFFF737FF002800D0AEE049
:10421000B36A002B41D022780C20029206321F2A6A
:1042200000D9A4E019880720052900D89FE0514A49
:104230008F18514ABFB2974200D898E05A88052A91
:1042400000D894E04B4FBF18BFB2BC464A4FBC45A4
:1042500000D88CE0494FB94204D0BA4202D0914212
:1042600000D984E0029A02990132227005226A5430
:104270002278511C21701221A95422781888A9187B
:104280000870000A4870901CC0B2207059882B1822
:1042900019700432090A59702270F76A002F28D069
:1042A0003A792378911C981CC9B241180C201F2917
:1042B0005DDC591C03322170EA5423785A1C2270A9
:1042C000FF22EA5423783988EA1802331170DBB2EE
:1042D000090A51702370BA88002A0AD0B9680720E9
:1042E000002944D0E81804F0ABFEBA882378D3182C
:1042F0002370371C34373B7800200397834236D035
:10430000316B814232D00290039F3B78029FBB42C7
:104310002AD9029A0C275743336BDF193A7923784D
:104320000332591C2170EA5423785A1C2270162239
:10433000EA5420783A882B1802301A70C0B2120A58
:104340005A702070BA88002A09D0B96800290DD0A7
:10435000281804F075FEBA882378D3182370029BBE
:104360000133DBB20293CFE7002000E0072007B063
:10437000F0BDC0467FF3FFFF7DF30000FFFF0000AC
:10438000F0B593B06D466E460023063507360C1C1B
:104390002B70337098420BD08388002B01D10720FB
:1043A00024E08368002BFAD01B785A07F7D516E073
:1043B000071C002C03D0A388002BF0D106E0221CA0
:1043C00029783378381CFFF7FDFD0FE0321C201CE4
:1043D0000AA9FFF765FE0AAA0028F1D006E002A9A3
:1043E0002A1CFFF75DFE02AF0028E2D013B0F0BD3B
:1043F00038B5041C081C0D1C04F00AFF6560208001
:1044000038BDA0DF7047A2DF70470000F0B593B061
:1044100003900191171C0293002904D1081C284A1B
:104420006D21FCF7DFFC002F04D1381C6E21244ADB
:10443000FCF7D8FC0BAC201C00211C22FBF7B8FEBB
:10444000237802221343012623706B469E75039B3B
:1044500000256A469382291C04A803226560E56052
:1044600025616561A561FBF7A3FE029A291C1378FB
:104470006A461374029A53786A465374937C0622F0
:10448000934302221343E7221340B3436A4606AE26
:104490009374301C1422FBF78BFE05AB0693019B33
:1044A00004AA3361074B72601888211C321C189BC8
:1044B00037817581B781FFF7A6FF13B0F0BDC04605
:1044C00082B20200542C0020F0B5624B89B005A9DD
:1044D000041C614A012088700B80FFF792FF0028BE
:1044E00000D0B4E02288002A03D12289002A16D005
:1044F0000AE05A4B5A480093231C61683C33FFF78B
:1045000085FF0028F1D0A2E0564B57480093231CAA
:10451000E1683C33FFF77AFF002800D097E0228A59
:10452000002A0AD0514B52480093231C61693C3346
:10453000FFF76CFF002800D089E0228B002A0AD008
:104540004C4B4D480093231CE1693C33FFF75EFF61
:10455000002800D07BE0228C002A09D0474B484835
:104560000093231C616A3C33FFF750FF00286ED193
:10457000228D002A09D0434B43480093231CE16A53
:104580003C33FFF743FF002861D1236B002B2FD072
:104590001A68FF2559682D02171C2F4003913F0A06
:1045A000684606A90A704776FF200004171C0740DA
:1045B0003F0CBC4666466F46BE76120E6F46039EA3
:1045C000FA7607AA16709B686A461D4053772D0A33
:1045D0006A46034095771B0C6A46D3772B4B2C48D1
:1045E0000093231C08223C33FFF710FF00282ED134
:1045F000636B002B20D1A06B002828D0037806A97C
:104600000B7043886A4653766A461B0A9376838802
:104610006A46D37607AA1B0A1370C3886A46537783
:104620006A461B0A93771B4A231C00923C330722DD
:104630001948FFF7EBFE0AE019681A79174B18487A
:104640000093231C3C33FFF7E1FE0028D3D009B0D0
:10465000F0BDC0460A180000542C00201C2C00207D
:10466000292A0000142C0020242A00003C2C0020C1
:10467000252A0000342C0020272A0000442C00208A
:10468000262A00000C2C0020282A00004C2C002098
:10469000232A00002C2C0020502A0000242C00206B
:1046A0002A2A000010B54378827801339A1A541EE2
:1046B000A241524213400278934206D00B604378E5
:1046C000182253434068C01800E0002010BD0000CD
:1046D000164B02205A68D205D20D26D0103AD3B21A
:1046E00059B200290DDA0F221A40083A1049C24087
:1046F00082405218032152680B408B40DA40131C51
:1047000008E08908C0310B4B8900CB5803210A40CF
:104710008A40D340DBB29B09DBB20020012B04D0DE
:10472000033B584243410220C01A704700ED00E0AD
:1047300018ED00E000E100E02F23C046C046C0466F
:10474000C046C046C046C046C046C046C046C04639
:10475000C046C046C046013B002BEED1704700006A
:1047600008B58022084B9202DA67D221074B8022DB
:10477000520289005A50C22189005A5001225A60BF
:10478000FFF7DAFF08BDC04604E100E00010014079
:10479000254AF8B5002353649364D36413655360CA
:1047A0009360224A1468621C3CD0214A21491E1C95
:1047B0008D58214A1268AD1A2D022D0A2422544325
:1047C0001E4B1A68121953689D4216D3ED1AF6183B
:1047D0001B4B146A1B689769D169002B09D0381CE0
:1047E0009847002807D0AA214900164AFCF7FAFA90
:1047F00001E0081CB847631CE0D1134B1978134B38
:104800001A788A4206D10132D2B21A70022A01D134
:1048100000221A701A780E4B9200D65080220D4B4F
:1048200052035A60F8BDC046FC100140702C0020B5
:104830000405000000100140582C0020602C0020CE
:104840005C2C0020B4B202006C2C00206D2C0020E7
:10485000742C0020FCE100E0F0B5CE4ACE4813688D
:1048600089B001680793CD4CCD4B0391247819781A
:104870008C4211D00131C9B2022900D10021197036
:104880001978C84B8900CC58039D012663191B0277
:104890001B0A0360059601E000240594C24B1B78B7
:1048A0000493C24B049F1B6800970193C04B186888
:1048B0001368009A013AD2B20092FF2A53D00099AD
:1048C000019ACD0055192A7869789142F1D01821C2
:1048D00051436E6801327118AE78D2B2B61A771EA3
:1048E000BE41764232400E78022E02D0032EEBD12A
:1048F00030E04F682421794341180291097DBC467C
:104900000029E1D0191C06934F1C1FD024276145B4
:1049100004D04F43C7190691396AF5E7069E8E42C7
:1049200002D17B43C3181B6A2427794341184E6880
:10493000096AB446069E7E43861931624E1C05D034
:10494000794341184F683E1C66444E60029E002128
:104950003175B9E75F1CB7D024214B430021C31840
:1049600019751B6AF6E78B4E05983360002809D14C
:1049700007995B1A5A1E9341DBB2039301235B42F2
:1049800000932DE08A4A00211268019201225242CE
:1049900000925A1C20D024225A43019DAA18506824
:1049A000844205D23360041B01265460039617E04D
:1049B000241A09180020506010751069176A002821
:1049C00008D0039DD0606D1800982D022D0A9560C7
:1049D000106200933B1CDCE76E4A136001230393D3
:1049E0006C4B1B680593714B1B680693704B1C68DE
:1049F000694BA4461B680293059B049A013AD2B204
:104A00000492FF2A7BD0049D069EE900711800984D
:104A1000013007D0009F24227A436244146A381C74
:104A2000009422E00A7848789042E6D01824544353
:104A30004D6801328878D2B22C190A70904201D1A7
:104A400000220A70227860681D1C012A55D1242298
:104A500042436244167D002E4FD1A6689660E768F7
:104A6000D760256915616469D461029F9568D4682F
:104A7000EE1B504F3602360ABE4201D8341908E008
:104A8000029E751B2D022D0AAC4201D9641B00E069
:104A90000024546000249460D4600124147564429E
:104AA00014622424251C454365445F1C24D05C43C8
:104AB00064446A686668B24202D901931C1C09E02A
:104AC000B21A62602B6217E0366AD21B771C0BD0D9
:104AD0000194341C2426664366447768BA42F3D8AE
:104AE000BF1A7760261C019C6A60242262436244DC
:104AF0002E6210621D1C00E0051C2B1C87E7254A56
:104B0000059913608B4202D1039A002A5ED05C1C87
:104B10005AD02421264A4B431268274CD3185F6889
:104B20001D4A264B1668E5580798AA1B1202120A5E
:104B300003320092013012D18023D1225B02920015
:104B4000A350C1229200A350C0211D4B802292028B
:104B500049005A501A6001232360FFF7EDFD009BC6
:104B6000BB4200D23B1C9B191B02A8221B0AD2008D
:104B70001249A35062585B1B521B1202120A1B02FD
:104B800003321B0A9A4221D980220E4B92025A60AC
:104B90001CE0C046702C0020582C00206D2C0020FA
:104BA0006C2C0020742C0020642C0020682C002029
:104BB000602C0020FEFF7F00001001400405000073
:104BC00000E100E0FCE100E0FFF7CAFD09B0F0BD44
:104BD000F7B5032401900E1C171C1D1C1C4054D15A
:104BE000002B52D0FFF7BCFD294B0898221C1860FF
:104BF000284B1E70284B1D602B1CB24205DA002189
:104C00001970197501322433F7E724235E43234AD0
:104C10000323182013707843214AAD1915602A1C0C
:104C200018320021013B6A6029706970AF70121858
:104C300008358B42F5D11B4A0121494211601A4ABD
:104C4000C0211370194A49001370194B8022520376
:104C50005A50C52189005858FF25A843C02528432C
:104C600058501A600198134AA121C9005050C4211C
:104C700089005D5810482840C0252D02284358500F
:104C80000E4BD2580E4B1A6000E00724201CFEBDCC
:104C90005C2C00206E2C0020602C0020642C002056
:104CA000682C0020702C00206C2C00206D2C002023
:104CB00000E100E000100140FF00FFFF04050000DC
:104CC000582C0020114BF0B51C68002C1AD0002A7B
:104CD0001AD0002818D00E4B1F780023BB420FDAE1
:104CE000251C2434261C243E3678002E06D10124AF
:104CF0002C706970AA610360301C06E00133EDE797
:104D0000042002E0082000E00720F0BD602C002015
:104D10006E2C0020F0B5204B85B001921A68051C5E
:104D20000C1C002A34D01D4B07201B789D4230D22A
:104D300004292ED924236B43D3181A780820012A7A
:104D400027D15B78012B01D0002700E00F1CFFF773
:104D5000BFFC134BC0001E6803A93618301CFFF7B8
:104D6000A1FC031C0420002B13D001221A700D4952
:104D70000D4A5D608A58DC609A60019A1F615A6131
:104D8000039B80227370094B52035A60002000E09D
:104D9000082005B0F0BDC046602C00206E2C00201D
:104DA000682C00200010014004050000FCE100E038
:104DB000154B37B51A68041C002A22D0134B1978FA
:104DC000072388421ED2242343439A5C0823012AE6
:104DD00018D1FFF77DFC0E4BC0001D6801A92D18EE
:104DE000281CFFF75FFC042300280BD0022303706C
:104DF000019B446080226B70064B52035A60002373
:104E000000E00823181C3EBD602C00206E2C002002
:104E1000682C0020FCE100E02BDF70472CDF70479E
:104E2000031C032010B5104010D1094C22604C1C0B
:104E3000E400A4B21219074C2260074A1070074A16
:104E40001070074A1380074B198000E0072010BD3F
:104E50007C2C0020802C0020872C0020862C002019
:104E6000842C0020882C0020F0B5464B85B00192A0
:104E70001A8800900C1C09208A4200D27FE06E46FE
:104E800000230F363370404B04275A68D205D20DE9
:104E900020D0103AD3B259B200290DDA0F221A40AD
:104EA000083A3A49920892005218032152680B407E
:104EB0008B40DA40131C08E08908C031344B89006C
:104EC000CB5803210A408A40D340DBB29B09DFB2B2
:104ED000012F0CD0301CFFF79FFF022801D172B6C2
:104EE00005E0002803D059212A4AFBF77BFF2A4B13
:104EF0002A4A18781188C0B20022884201D2421C86
:104F0000D2B22748007882420BD01D781A78EDB2D1
:104F1000D2B200238A4201D2531CDBB21E4A137064
:104F200000E0204D012F0BD062B63078FFF776FFFE
:104F30000223021C9A4303D06121164AFBF752FF59
:104F4000184B04209D421AD0174FEE003968019A81
:104F50008B1900991A6000290FD0002C0DD0094A36
:104F6000124B1088221C45431868401904F068F859
:104F70003B6800209E19B48001E00020988005B0B5
:104F8000F0BDC046842C002000ED00E018ED00E0EC
:104F900000E100E0E2B20200872C0020882C002013
:104FA000862C0020FFFF00007C2C0020802C00209D
:104FB00010B5104B1978104B1A78914219D00F493F
:104FC0001A7818780C88C0B2D2B20021844201D974
:104FD000411CC9B219700A49D3000968CB180949A4
:104FE0000888094942430868998880181B689847CF
:104FF000DFE710BD872C0020862C0020882C0020A5
:105000007C2C0020842C0020802C002075DF704731
:1050100076DF70477ADF70477BDF7047174B37B515
:105020001888174B984227D0164B174D1A78297BB2
:105030000132D2B21A702C1C914208D31349FFF7E7
:10504000E5FF002818D0AB69002B14D114E0002232
:105050001A702B7C934208D03B21FFF7D9FF002820
:1050600003D0AB69002B00D098476369002B03D0B5
:1050700001A800220270984737BDC046B82C002016
:10508000FFFF0000942C0020982C0020BA2C002058
:1050900037B5184B184A5B881188184C184D99423F
:1050A0000CD852889A4209D36369002B03D001A817
:1050B00001220270984700232B7037BD2B78002BFC
:1050C00005D06369002BF6D001A80022F1E70D4B53
:1050D0001B78002B01D1616800E0A1680A4B002217
:1050E0001868FFF717FE0028E5D0A369002BE1D16F
:1050F000E1E7C0468C2C0020BA2C0020982C002020
:105100008A2C0020942C0020B42C002070B5144967
:10511000021C0B1C70CA70C332CA32C31268114C15
:105120001A600168104B00221A70201C914213D0A3
:10513000082203F085FF201CFFF76CFF00280ED12A
:105140000A4B012252421A80094B0021094A0A489F
:105150001970FFF7B7FD02E0FFF75EFFEEE770BDE5
:10516000982C0020BA2C00208A2C0020B82C00207B
:10517000942C00201D500200B42C002010B5038890
:10518000112B19D002D8102B05D043E0122B3AD0A6
:10519000502B21D03EE082881F4B011C1A800E311B
:1051A00008221E4803F04CFF1D4B00221A701D4BB5
:1051B000DB8993422ED12BE0174B012252421A80F9
:1051C000174B00221A70184B1868FFF7F1FD0028E2
:1051D00020D0144B9B6912E0124CC188E2899142A5
:1051E00018D1C38B022B15D10130C37FDA070FD43E
:1051F0000D4B1868FFF7DCFD00280BD0A369002BCE
:1052000008D0984706E0811D0822044803F018FFE3
:10521000FFF73EFF10BDC046B82C00208C2C0020AC
:10522000942C0020982C0020B42C002051DF7047D3
:1052300050DF704737B5094B021C197814204143E1
:105240005C18E068217905016369201CE4880C3052
:105250000094034C2C59A04737BDC046C42C0020F5
:10526000202F0020F7B5634C00932378061C0F1CF9
:10527000151C002B06D1009B134301D1022300E033
:105280000123237023780320013B052B00D9B0E0D4
:10529000181C00F097FB032334557E91564A802357
:1052A00051695B05013105D05069196989B200F077
:1052B00093FB00E0586980235B051D6919691A6931
:1052C0000138ABB289B292B2584379439208FFF7E2
:1052D000ADFF0223002800D18AE08AE0381CFFF7E6
:1052E000A7FF002800D084E00323002D00D07FE03A
:1052F0000099002922D13378042B48D177E080230C
:105300005B051A6992B257433B4A5169013105D096
:105310005069196989B200F05FFB00E05869802389
:105320005B051969013889B241432A1C381CFFF713
:105330007DFF00285DD1009A002A25D0042357E084
:1053400080235B051A69718892B257432A4A7F18F5
:1053500001915169AD007F19013105D0506919697A
:1053600089B200F039FB00E0586980235B051969B8
:10537000013889B24843019AAD182918009A381C9F
:10538000FFF754FF002834D13378042B12D00523C3
:105390002EE080235B051869728880B24743AB001A
:1053A000D81931699208FFF741FF002821D1009BED
:1053B0001D431CD006231BE00F4A802351695B0567
:1053C000013105D05069196989B200F005FB00E090
:1053D000586980235B051A691969013893B25843EB
:1053E00089B200F0F9FAFFF723FF002801D1072363
:1053F0002370FEBD492F002000100010F8B5324E7A
:10540000142233785343F3181C1D1B79E568042BD1
:1054100018D0052B39D00F20022B54D12B4B62888A
:105420001888236980021918A388121A5D19284B5D
:1054300028189A4201D8920801E080225200FFF712
:10544000F5FE3CE0A26823491301CB18198958895D
:105450005B6880277F05AB4203D141436388994253
:1054600001D0032A0AD13969281C89B200F0B4FAA4
:10547000164B1B88C018FFF7DBFE20E03969281C9B
:1054800089B200F0A9FA011C09E080277F0539697B
:10549000281C89B200F0A0FAA388011C5D193A69A2
:1054A0003B6992B2481C4A439BB243436088AA1AA4
:1054B00045195B1B92089B08201CFFF7D3FE0028B0
:1054C00001D10123B370F8BDC42C00204A2F002065
:1054D000FF030000202F0020F8B5134C061C657850
:1054E00006A8078804201E2D1DD020782D18EDB2A7
:1054F0001D2D01D91E3DEDB21420454365196A6189
:105500002A1C2E710C3241C941C2EB802F81A37835
:10551000002B01D0002003E0FFF770FF1128F9D025
:10552000637801336370F8BDC42C002010B5074BBD
:1055300000245B78A34207D0FFF760FF041E03D06E
:10554000112801D0FFF776FE201C10BDC42C0020CE
:10555000F0B53E4A87B09378141C002B74D03C49B8
:10556000002393700A78082A06D1022801D10B7013
:1055700064E0384A137061E0022803D0032863D145
:105580000D205FE0217814204843334D2018011D81
:105590008C4629880079013189B20191298002283D
:1055A0000AD18E02614649880296029FF517CE0FF6
:1055B0008F426E41059607E0052804D1D51F6E4243
:1055C0007541059301E005931D1C04280BD1D31FE1
:1055D000584243410198664681027088814205DB4A
:1055E00051424A4103E000231A1C00E00022002D32
:1055F00007D1002B05D1002A03D1059F01231F42AB
:105600001CD0134800250570281CFFF713FE2278D4
:10561000142353430221E3181D71DD80D9601D61FD
:105620005D611D8163780C4E013B6370531CDBB2DE
:10563000358023701D2B01D91D3A2270FFF776FFAC
:10564000002801D0FFF7F6FD07B0F0BDC42C002004
:10565000492F0020482F00204A2F002038B52C4A1F
:105660002C4C0023138023706370A370191C6218E4
:10567000002302201371D380D06013615361138122
:105680001431962282409142F1D1234A234D138056
:105690006A6980235B05013205D06869196989B29E
:1056A00000F09AF900E05869802149050B69033838
:1056B0009BB258431A4B002218601A4B1A601A8189
:1056C0009A815A811A611A839A835A83164B082247
:1056D0001A706B69013306D0104B5869096989B299
:1056E00000F07AF900E0486980235B051A691969BE
:1056F000013893B2584389B200F06EF9FFF798FD74
:10570000002803D1094A0123A370137038BDC04695
:105710004A2F0020C42C0020402F00200010001031
:10572000442F0020202F0020492F0020482F002048
:10573000F0B5384B85B01B780E1C0822002B66D0C4
:10574000002863D0002961D00168039100295DD051
:1057500080235B051969858889B207228D4256D856
:105760000F2D54D9C0880190002850D0041C2A4A1B
:105770006C4312680292A718284A5169013105D07A
:105780005069196989B200F027F900E0586980234F
:105790005B051B6901389BB258430722874236D804
:1057A00003272F4033D11E4A138894460422022B2C
:1057B0002DD0029A180172601A4A3360029E1118A5
:1057C0004E60039E8650019E0D814E8112490868ED
:1057D0000D1C802149050E690137B6B2BFB2B44233
:1057E00003D90E69B6B2A41B00E000240E69096952
:1057F000B6B289B280198C42EBD2190152182860D6
:105800000133604697810380002200E00E22101CC5
:1058100005B0F0BD482F0020442F002000100010DC
:10582000402F0020202F0020F0B5141C1D4A051C1D
:10583000127885B00E1C0820002A30D000292DD007
:10584000002D2BD029680720012928D8164A0901E4
:105850008F58002F23D06F68511803970A894F89FA
:1058600049685743BC46039F61448F4217D2002CBE
:1058700015D0944213D8E118914210DC0322102075
:1058800016420CD113420AD1174208D10093291CA9
:10589000321C231C0220FFF71FFE00E00E2005B083
:1058A000F0BDC046482F0020202F0020F8B51A4C2C
:1058B00025780824002D2DD000292AD0002828D0B2
:1058C0000E680724012E25D8144D36017759002F74
:1058D00020D0AE193589778949686F43BC4677680F
:1058E0006744B94216D2002A14D0AA4212D8D61858
:1058F000AE420FDC0325102428420BD12B4209D1E4
:105900002C1C0C4003D1591803F09AFB02E0102420
:1059100000E00E24201CF8BD482F0020202F00207E
:10592000164B73B51B78041C0D1C0820002B24D0CB
:10593000002C21D022680720012A1ED8104912010C
:105940005358002B19D08A185668118952896368F8
:105950004A439219934210D210209A070DD1981BF6
:1059600000F07EF807200A1E07D100912B1C211C95
:105970000420FFF7B1FD00E00E2076BD482F002087
:10598000202F002082B00190019B002B15D0019B9D
:10599000013B01930A4BC046C046C046C046C046C4
:1059A000C046C046C046C046C046C046C046C046C7
:1059B000C046013B002BEED1E6E702B07047C0467F
:1059C000E703000002B4714649084900095C490038
:1059D0008E4402BC7047C046002934D00123002207
:1059E00010B488422CD301242407A14204D281425E
:1059F00002D209011B01F8E7E400A14204D281426E
:105A000002D249005B00F8E7884201D3401A1A43EA
:105A10004C08A04202D3001B5C0822438C08A04221
:105A200002D3001B9C082243CC08A04202D3001BD7
:105A3000DC082243002803D01B0901D00909E3E751
:105A4000101C10BC7047002801D00020C04307B4D0
:105A5000024802A14018029003BDC046D9000000D0
:105A60000029F0D003B5FFF7B9FF0EBC4243891AF5
:105A70001847C046002941D010B4041C4C40A4462D
:105A800001230022002900D54942002800D54042C8
:105A900088422CD301242407A14204D2814202D29D
:105AA00009011B01F8E7E400A14204D2814202D2BD
:105AB00049005B00F8E7884201D3401A1A434C08BA
:105AC000A04202D3001B5C0822438C08A04202D3F0
:105AD000001B9C082243CC08A04202D3001BDC0818
:105AE0002243002803D01B0901D00909E3E7101C59
:105AF0006446002C00D5404210BC7047002806D0F8
:105B000003DB0020C043400801E08020000607B40A
:105B1000024802A14018029003BDC04619000000CF
:105B20000029EBD003B5FFF7A7FF0EBC4243891A4B
:105B30001847C0467047C0468446081C6146FFE7C8
:105B40001FB500F0C5FB002801D40021C8421FBDCD
:105B500010B500F04DFB4042013010BD10B500F013
:105B6000B7FB002801DB002010BD012010BDC0469E
:105B700010B500F0ADFB002801DD002010BD0120B4
:105B800010BDC04610B500F05BFB002801DC002012
:105B900010BD012010BDC04610B500F051FB00281B
:105BA00001DA002010BD012010BDC046002B11D12C
:105BB000002A0FD1002900D1002802D00021C943BA
:105BC000081C07B4024802A14018029003BDC04659
:105BD00065FFFFFF03B4684601B5029800F05CF86A
:105BE000019B9E4602B00CBC7047C0469E2110B57A
:105BF000C905041CFFF7D0FF002803D1201C00F0CA
:105C000051FE10BD9E21C905201C00F0D5FC00F0FE
:105C100049FE80231B06C018F3E7C04600000000C1
:105C200038B50E4B0C4A041C0D1C02F0D3FC0028A6
:105C300004D1201C291C02F015FB38BD074B064A75
:105C4000201C291C01F0D8FF02F00CFB80231B064E
:105C5000C018F2E7C046C046000000000000E04166
:105C6000F0B583B0161C1F1C0090019102F0FCFCE3
:105C7000041C0D1C221C2B1C301C391C02F0D2FCF5
:105C8000009A019B121A8B410899201C0A604B60F4
:105C9000291C03B0F0BDC046F0B583B0141C1D1C18
:105CA0000090019102F0B8FE221C2B1C061C0F1C58
:105CB00002F0B8FC009A019B121A8B410899301C23
:105CC0000A604B60391C03B0F0BDC046F8B5430212
:105CD0004400C50F4E024800240E2A1C9B09000EEA
:105CE000C90FB6098D425BD0221A002A00DC89E078
:105CF00000281DD1002E00D075E0580704D00F22D7
:105D00001A40042A00D004338021C90419402A1CF7
:105D100000293AD00134FF2C00D17FE09B015B0ABF
:105D20005B02E4B2E405580AD20720431043F8BDF1
:105D3000FF2CE2D08021C9040E431B2A00DD2BE199
:105D4000311C2020D140821A9640721E96410E438B
:105D50009B1B5801D1D59B019F09381C02F044FCC4
:105D6000421F974094425BDC141B1F231B1B3A1CF1
:105D70009F40611C3B1CCA405F1EBB411343002473
:105D8000BBE7131EB9D100230022DB08FF2C04D18E
:105D9000002B43D08020C00303435B025B0ABFE7B4
:105DA000211A002940DD002823D0FF2CA5D0802017
:105DB000C00406431B2900DDECE0301C2027C8404E
:105DC000791A8E40711E8E4106439B19590100D4E9
:105DD00093E70134FF2C55D0704901221A400B4043
:105DE0005B08134389E7013A002AB1D0FF2CA4D104
:105DF00083E7002E00D180E701390029E5D0FF2C90
:105E0000D8D17AE7002A1BD1621CD2B2012A4ADD1E
:105E10009F1B7A0123D5F71A0D1C9EE700237FE70D
:105E20005E4BA41A3B4068E7002945D1611CC8B20B
:105E3000012829DDFF2924D0F3185B080C1C5CE73E
:105E4000002C13D0FF2818D08024E40452422343AE
:105E50001B2A4CDD0123F31A041C0D1C79E7002FCB
:105E600000D07AE70023002200248EE7002B3AD0EE
:105E7000D243002AEFD0FF28EAD1331CFF240D1CA7
:105E80003BE7FF24002380E7002C5BD1002B7FD071
:105E9000002E00D131E79B19580100D42DE73F4A6D
:105EA0000124134029E7002C15D1002B40D1002EEE
:105EB00062D0331C0D1C20E7002C21D1002B54D0C4
:105EC000C943002904D0FF284CD01B2957DD0123EA
:105ED0009B19041C7AE7002B19D1002E48D0331CE3
:105EE0000D1CFF2409E7331C041C0D1C05E71C1CBA
:105EF0002025D440AA1A93405A1E93412343AAE76F
:105F0000FF282FD08024E40449422343DDE7FF2407
:105F1000002E00D1F1E68022DB08D203134204D028
:105F2000F608164201D1331C0D1CDB00FF24E4E609
:105F3000002E00D1E1E69A1B500100D421E7F31AAC
:105F40000D1CDAE6002B0DD0FF24002E00D1D4E684
:105F50008022DB08D2031342E7D0F6081642E4D1D0
:105F6000331CE2E7331CFF24C7E6331C041CC4E6E1
:105F700000220B4BFF2408E7231C002205E71C1C12
:105F80002027CC40791A8B40591E8B4123439FE731
:105F9000331CB2E6012618E70126D9E6FFFFFFFB16
:105FA000F8FFFF03F0B55F4656464D464446F0B451
:105FB00046024500C00F85B00F1C760A2D0E8046A4
:105FC00041D0FF2D26D08024240400212643F60052
:105FD0007F3D89468B46F90F7C027800640A000EEB
:105FE00000918A463CD0FF2834D080231B041C43F8
:105FF0000023E4007F380193009F4346019A7B40D1
:1060000049469C4611430F2900D970E0754F89001D
:106010007F58BF46002E3ED10822022391469B4660
:10602000D9E75A46341CC24601920199022937D059
:10603000032900D1CEE0012900D0AAE053460B404D
:106040000022002632E0002E19D1042101228946C7
:106050009346C0E7221C531E9A4102320192CBE7BD
:1060600001270197002CC7D0201C02F0BDFA431F66
:106070009C4076235B420021181A0191BCE7301C3A
:1060800002F0B2FA7625431F9E406D4200232D1A7E
:1060900099469B469FE70C23032199468B469AE736
:1060A000D446012367463B40FF2200267602D205F4
:1060B000700ADB071043184305B03CBC9046994674
:1060C000A246AB46F0BD0023474EFF22EEE700227A
:1060D0000026EBE78020C00306423BD0044239D1C2
:1060E000061C26437602760A009BFF22DEE7281A6A
:1060F000039076016401A64239D3361B1A2201238C
:106100000120311C5B007600002901DBB44201D87C
:10611000361B0343013A002AF3DC741EA641341CEB
:106120001C43039A7F32002A27DD630704D00F2324
:106130002340042B00D00434270103D52B4B039AB2
:106140001C408032FE2A0BDD012361460B40FF22FA
:106150000026ABE706437602760A4346FF22A5E710
:10616000A40101236746660AD2B23B409EE7039F23
:106170001B22013F03970023C2E77E23039F5B425C
:10618000DB1B1B2B07DD012361460B400022002691
:106190008CE7D446C5E7221CDA40039B9E339C4023
:1061A000231C5C1EA34113435A0704D00F221A403C
:1061B000042A00D004335F0105D5012361460B405A
:1061C0000122002672E79E01624601231340760AEF
:1061D00000226BE78026F60326437602760A5346B2
:1061E000FF2263E714B30200FFFF7F00FFFFFFF70A
:1061F0004A02430270B55C0A550A43004A001B0E6E
:10620000C60F120EC90FFF2B05D0FF2A08D00120A0
:1062100093420BD070BD0120002CFBD1FF2AF6D198
:106220000120002DF6D101209342F3D1AC42F1D1EF
:106230008E4203D0002BEDD1002CEBD10020E9E7FA
:106240004A024302F0B55C0A550A43004A001B0E9D
:10625000C60F120EC90FFF2B26D0FF2A29D0002B04
:106260000CD1604260418446002A0AD0002816D131
:106270008E4221D0002E14D1012014E0002AF7D143
:1062800094466F426F416046002805D1002FEFD041
:106290000120002E07D004E00020002F03D10029A8
:1062A000EAD101204042F0BD002CD6D0022040426D
:1062B000F9E7002DD3D0F9E79342DBDC04DBAC42F5
:1062C000D8D80020AC42EED2002EEAD00120EAE776
:1062D0004A024302F0B55C0A550A43004A001B0E0D
:1062E000C60F120EC90FFF2B26D0FF2A28D0002B75
:1062F0000FD0002A14D194466F426F4160460028A7
:1063000014D00020002F03D100290DD101204042DC
:10631000F0BD604260418446002AEDD00028F3D1F0
:106320008E4211D0002EF1D10120F1E7002FF7D0DD
:106330000120002EECD0E9E70220002CE8D1D4E7C0
:106340000220002DE4D1D2E79342EBDC04DBAC4227
:10635000E8D80020AC42DBD2002ED7D00120D7E70E
:10636000F0B55F4656464D464446F0B444024600FA
:1063700083B00F1C640A360EC50F002E41D0FF2ECD
:1063800022D080231B0400201C43E4007F3E824671
:106390008046391C4B007F02C90F7F0A1B0E8B46BB
:1063A0003BD0FF2B34D0802212041743FF007F3BE9
:1063B00000215A466A40019252460A430F2A62D887
:1063C0007A48920082589746002C3FD10822022337
:1063D00092469846DDE70195404602282AD1019A67
:1063E00001251540FF2300246402DB05600AED0748
:1063F0001843284303B03CBC90469946A246AB469E
:10640000F0BD002C27D10420012282469046C0E72F
:10641000391C4A1E91410231CBE70121002FC8D01F
:10642000381C02F0E1F8431F9F4076235B421B1AA1
:106430000021BEE7032800D1ADE001284ED101982C
:1064400042461040C5B200230024CDE70C230320B0
:106450009A4680469DE7201C02F0C6F87626431F28
:106460009C4076420023361A9A46984691E70025CA
:106470004F4CFF23B8E75B463C1C01938846ABE7D3
:106480003C1C8846A8E7250C24043A0C240C3F0445
:10649000F6183F0C211C231C794353436F4355438B
:1064A000FB180A0C9B18B1469F4202D98022520267
:1064B000AD1809041A04090C521894011B0C611E32
:1064C0008C41920EED181443AD012C43230105D5E8
:1064D000012263080120144081441C434B467F3352
:1064E000002B2DDD600704D00F222240042A00D0AB
:1064F0000434220103D52F4B1C404B468033FE2B26
:1065000017DD019B01251D400024FF236CE780203F
:10651000C003044208D0074206D1041C3C43640275
:10652000640A5D46FF235FE704436402640AFF23B5
:106530005AE70198A4010125640ADBB2054053E73C
:106540007E235B424A469B1A1B2B05DD019B0125DE
:106550001D400024002347E7221CDA404B469E33AF
:106560009C40231C5C1EA3411343580704D00F22F8
:106570001A40042A00D004335A0105D5019B012595
:106580001D40002401232FE701989C010125640A86
:106590000540002328E78027FF03019B3C4364025A
:1065A00001251D40640AFF231EE7C04654B30200C4
:1065B000FFFF7F00FFFFFFF7F8B5C20F4302440063
:1065C0004D024800240E161C9B09000EC90FAD0990
:1065D000FF2800D183E0012779408A425CD0221A4B
:1065E000002A00DC8EE000281ED1002D00D07AE0C9
:1065F000580704D00F221A40042A00D00433802107
:10660000C90401221940324000293AD00134FF2C3C
:1066100000D183E09B015B0A5B02E4B2E405580A07
:10662000D20720431043F8BDFF2CE1D08021C904DC
:106630000D431B2A00DD2FE1291C2020D140821AA6
:1066400095406A1E95410D435B1B5801D0D59B01B7
:106650009F09381C01F0C8FF421F974094425FDC3D
:10666000141B1F231B1B3A1C9F40611C3B1CCA4070
:106670005F1EBB4113430024BAE7131EB8D10023A9
:106680000022DB08FF2C04D1002B47D08020C00360
:1066900003435B025B0ABFE7211A002944DD00289F
:1066A00027D0FF2CA4D08020C00405431B2900DD87
:1066B000F0E0281C2027C840791A8D40691E8D41C2
:1066C00005435B19590100D492E70134FF2C59D0DE
:1066D000724901221A400B405B08134388E7002DE2
:1066E00000D07AE777E7013A002AADD0FF2CA0D19D
:1066F0007EE7002D00D17BE701390029E1D0FF2C96
:10670000D4D175E7002A1BD1621CD2B2012A4ADD1E
:106710005F1B7A0123D5EF1A0E1C9AE700237BE753
:106720005E4BA41A3B4063E7002945D1611CC8B207
:10673000012829DDFF2924D0EB185B080C1C57E742
:10674000002C13D0FF2818D08024E40452422343A5
:106750001B2A4CDD0123EB1A041C0E1C75E7002FCD
:1067600000D076E70023002200248AE7002B3AD0ED
:10677000D243002AEFD0FF28EAD12B1CFF240E1CA5
:1067800036E7FF2400237CE7002C5BD1002B7FD071
:10679000002D00D12CE75B19580100D428E73F4AAF
:1067A0000124134024E7002C15D1002B40D1002DEB
:1067B00062D02B1C0E1C1BE7002C21D1002B54D0C7
:1067C000C943002904D0FF284CD01B2957DD0123E1
:1067D0005B19041C76E7002B19D1002D48D02B1C27
:1067E0000E1CFF2404E72B1C041C0E1C00E71C1CC1
:1067F0002026D440B21A93405A1E93412343AAE75D
:10680000FF282FD08024E40449422343DDE7FF24FE
:10681000002D00D1ECE68022DB08D203134204D025
:10682000ED08154201D12B1C0E1CDB00FF24DFE616
:10683000002D00D1DCE65A1B500100D41DE7EB1AF5
:106840000E1CD5E6002B0DD0FF24002D00D1CFE685
:106850008022DB08D2031342E7D0ED081542E4D1D1
:106860002B1CE2E72B1CFF24C2E62B1C041CBFE6FA
:1068700000220B4BFF2404E7231C002201E71C1C11
:106880002027CC40791A8B40591E8B4123439FE728
:106890002B1CADE6012514E70125D5E6FFFFFFFB24
:1068A000F8FFFF034302590A4300C20F1B0E0020EA
:1068B0007E2B0DDD9D2B0CDC802000040143952BED
:1068C0000ADC9620C31AD9404842002A00D1081C8D
:1068D0007047034BD018FBE7963B9940F4E7C0465E
:1068E000FFFFFF7F70B5041E3CD0C60F00D04442AE
:1068F000201C01F079FE9E23251C1B1A962B0CDC14
:10690000083884406402640ADBB2321C6402DB058E
:10691000600AD2071843104370BD992B0ADD052287
:10692000121A211CD1400A1C011C1B318D40691E0A
:106930008D411543052801DD421F9540164C2C4022
:106940006A0704D00F221540042D00D004346101E1
:106950000CD59F23181AFF281AD0A401640AC3B2C9
:10696000321CD3E7002200230024CFE7E408FF2BEA
:1069700004D06402640ADBB2321CC7E7002C04D0E6
:106980008020C00304436402640A321CFF23BDE775
:10699000321CFF230024B9E7FFFFFFFB10B5041EE4
:1069A00033D001F021FE9E231B1A962B09DC0838F8
:1069B00084406402640ADBB26402DB05600A1843A7
:1069C00010BD992B0ADD0522121A211CD1400A1C88
:1069D000011C1B318C40611E8C411443052801DDD4
:1069E000421F9440144A2240610704D00F210C40FA
:1069F000042C00D0043251010AD59F23181AFF2815
:106A000016D09401640AC3B2D6E700230024D3E76A
:106A1000D208FF2B03D05402640ADBB2CCE7002A71
:106A200006D08024E40314436402640AFF23C3E70E
:106A3000FF230024C0E7C046FFFFFFFBF8B55F4619
:106A4000564644464D46F0B40C034D00CE0F610A45
:106A5000440F2143C400180380465800400D82466D
:106A6000D80F84464046400A530F0343D0006D0DB3
:106A7000371C83465246664500D1A4E0AF1A002F6A
:106A800000DC09E1002A3BD1184300D0EAE06307AB
:106A900000D187E00F232340042B00D182E0221D88
:106AA000A242A4416442802309191B040B40371CF5
:106AB000141C002B00D17CE0CE4B01359D4200D14F
:106AC00005E1CD4BE40819404807490204430B0B8C
:106AD000002000211B031A0B0B0D6D051B05134332
:106AE0006A08C64DFF071D4015436D006D08291C3F
:106AF0003943201C3CBC90469946A246AB46F8BDA3
:106B0000BC488542C3D0802000040343382F00DDF9
:106B1000F0E01F2F00DD24E12020C01B1A1C81465D
:106B200082405846F8400243944658464A469040B0
:106B3000421E9041FB40624602431F1CA21A94422F
:106B4000A4416442C91B091B141C0B029FD54902B6
:106B50004F0A002F00D1C8E0381C01F045FD021C8F
:106B6000083A1F2A00DDB5E02821091A201C9740A9
:106B7000C84007439440954200DDB2E0551B691CB4
:106B80001F2900DDDCE01F22551B3B1C221CAB40F3
:106B9000CA40AC40651EAC411343CF401C43391C76
:106BA000002574E780231B040B40371C002B00D00A
:106BB00082E7904B4807E4080443C9089D4248D047
:106BC00009030B0B84E7AA1A9446002A00DC98E01C
:106BD0005046002852D08748854200D157E7802090
:106BE000000403436246382A00DDFCE01F2A00DD72
:106BF0004AE120226046101A1A1C824082469146C1
:106C000058466246D0404A4602439046584652464D
:106C10009040421E9041424602436046C3401219D2
:106C2000A242A441644259180919141C080200D454
:106C30002DE7704B01359D4200D122E16E4B60087B
:106C40001940012323401C1C0443CB071C43490863
:106C50001DE7231C0B433AD080231B030B431B036C
:106C60001B0B35E7013F002F65D15846221A94428D
:106C7000A4416442C91A091B141C66E7584618430C
:106C800000D104E70122524294446046002800D01B
:106C9000C5E058460219C3E7002F73D1681C4005B0
:106CA000400D012800DCDEE05A46A21A9442BF41A2
:106CB000C81A7F42C71B380200D489E05A46141B09
:106CC000A3459241591A52428F1A664641E7002362
:106CD0000024FDE6271C283887400024954200DC6C
:106CE0004CE74549AD1A3940D1E6201C01F07CFC47
:106CF000203034E75A461A43531E9A41D2B2002735
:106D00001CE7002A00D0DCE0681C4205520D012A75
:106D100000DC8DE0374DA84200D1F3E05D462A1932
:106D2000A242A441644259180919CC0752081443DD
:106D30004908051CABE62F48854200D0E6E6A6E6EA
:106D40002B1C1F3B3A1CDA40131C20296CD03F221D
:106D5000551BAF403C43601E84411C43002100256D
:106D600095E6381C20381A1CC240101C202F5DD01C
:106D70004022D71BBB405A461A43531E9A41024336
:106D80000027DBE6002D3BD01A4DAA4500D193E049
:106D900080252D047F422943382F00DDACE01F2FD2
:106DA00000DD29E12025ED1B081C261CA840FE4023
:106DB000AC400643651EAC413443F9405D462C1B94
:106DC000A34592415B1A5242991A55466646BCE663
:106DD000131C3B43141C002B00D0BAE600270021F3
:106DE00000240025E5E65A461A43531E9A41D2B2C2
:106DF000002314E7FF070000FFFF7FFFFFFF0F8066
:106E00000D1C254358D0FF43002F51D1041BA3452F
:106E10009241591A5242891A5546664695E6964855
:106E2000854200D0DEE632E6002793E70023A2E7A2
:106E3000081C2043002D00D0C4E0002800D1F7E05A
:106E40005846184300D122E658460219A242A441EE
:106E5000644259180919141C0A0200D417E6874B1A
:106E60000125194013E6081C2043002D39D10028C4
:106E700071D15946194303D0191C5C46664606E693
:106E800000270021002494E6604620381A1CC240E6
:106E900060469146202800D1ACE04022121A93406F
:106EA0005A461A43531E9A414B461A430023B6E6EC
:106EB000714DAA4500D06FE7191C5C4655466646E1
:106EC000E5E5002D22D10D1C254377D0D543002DBB
:106ED00071D15C445C45924159185242891855461B
:106EE000A4E600284DD15946194300D194E0191C5D
:106EF0005C466646604DCAE50C43611E8C41E4B2B7
:106F000000215BE7051C0021002452E65A4DAA45EA
:106F100054D05542802210040143382D00DD81E019
:106F20001F2D00DD92E02022501B0A1C8446824067
:106F3000201CE8400243904662469440601E844113
:106F400042461443E9405C445C459241CB185242AE
:106F5000991855466AE65846184300D197E55846B1
:106F6000271ABC429241C81A5242801A020266D5C0
:106F70005846041BA3459241591A5242891A664643
:106F800085E55846184333D04807E4080443802079
:106F9000C9080003014208D0DD08054205D1594661
:106FA000CA085C071443291C6646630FC9001943CD
:106FB000E400314D6BE5304A9245AED1191C5C4678
:106FC000554664E5002836D05846184310D0802531
:106FD0004807E408C9082D0304432942E5D0D8082E
:106FE0002842E2D15D46EA085C071443011CDCE755
:106FF000214D4CE5002353E73D1C203D0A1CEA408F
:10700000151C202F34D04026F71BB9400C43611EBD
:107010008C412C430021D1E6082400271849644202
:10702000154DC6E50C43611E8C41E4B200218AE790
:10703000191C5C462BE5191C5C460F4D27E5031C0B
:107040003B4300D11CE7011C3C1C20E520204042B2
:1070500040190A1CC2409046202D0BD04020451BF1
:10706000A9400C43611E8C4145462C4300216AE730
:107070000021CBE70021F4E7FF070000FFFF7FFFBF
:10708000FFFF7F00F0B5564644465F464D46F0B4DC
:107090001F1C0B031B0B98464B0087B0041C81463A
:1070A0005B0DC80F161C9A460090002B51D06B4BFD
:1070B0009A4531D08022414652030A43630FD200E1
:1070C0001A43674B90460025E20091469A440024FB
:1070D00002953B031B0B9B46FD0F7B00311C5B0D98
:1070E000019560D05D4A934254D0802158464903AF
:1070F0000143720FC9001143594A8B469B18F10096
:107100000020009A04436A4003920F2C00D9B1E09A
:10711000544EA4003459A746404604436ED1002182
:1071200002250824884689460295D2E7009C0298E9
:10713000C34649460194022864D0032800D1AFE237
:10714000012800D03CE2019A002402400025A1461B
:1071500060E0434623434AD04046002800D1C4E1C2
:1071600001F042FA031E272B00DDB7E128210D1A9A
:10717000211C083B4246E9409A400D1C1543221C45
:107180009A40A8469146384B00251B1A9A4600247F
:1071900002959EE75A4616430320002EB1D1B3460E
:1071A00000210220ADE75A4632431BD05B46002B3C
:1071B00000D18EE1584601F017FA272800DD81E161
:1071C0002822171A011C321C08395B46FA408B40F2
:1071D000171C1F43331C8B40BB46191C224B1B1A28
:1071E00000208EE70027BB460021012089E7002010
:1071F000012504248046814602956AE703250C2474
:10720000029566E7019C0394039D01222A40002415
:10721000124DA146002000212403260B0C0D24054D
:10722000124B34432D0523402B435B005B08D207F0
:10723000191C4846114307B03CBC90469946A246EB
:10724000AB46F0BD01235B420022094C9946034D39
:10725000E0E700240025A146DCE7C046FF07000068
:1072600001FCFFFF94B302000DFCFFFFFFFF0F8046
:10727000FFFF0F005546ED1A0495D84500D953E19C
:1072800000D14EE1049C0025013C4E460494474643
:10729000A946584603020C0E1C430902250C230480
:1072A0001B0C0091381C291C0193FEF795FB0199DA
:1072B00083464143381C8A46291CFEF7D1FB330C18
:1072C000090419438A450CD95B460919013B8C42D4
:1072D00000D947E18A4500D844E102225242934452
:1072E00009195346CB1A181C291C9846FEF774FB43
:1072F000071C0198291C784382464046FEF7B0FBE4
:1073000036040B04360C33439A4509D91B197A1EEF
:107310009C4200D924E19A4500D821E1023F1B1983
:107320005E4632041743380CBB46009E009F514610
:107330003F0C32045B1A5946BA46120C0F043F0C3C
:10734000904651467A434F43414641435646704327
:10735000CF19160CBE19B14202D980277F02C0197D
:10736000310C12043604120C4018B618834200D2B5
:10737000C4E000D1BEE0191A4846861BB145BF41A2
:107380007F42CF1BA74200D113E1291C381CFEF716
:1073900023FB019902904143381C8946291CFEF7C2
:1073A0005FFB330C0904194389450CD9029B091969
:1073B000013B8C4200D9FFE0894500D8FCE0029FE8
:1073C0000919023F02974F46CF1B381C291C05970D
:1073D000FEF702FB071C0198291C7843814605989B
:1073E000FEF73EFB36040904360C0E43B14509D9BD
:1073F00036197B1EB44200D9E0E0B14500D8DDE08B
:10740000023F3619029D4946761A290439430B0476
:1074100057460A0C1B0C40464546584355437B4390
:107420007A43EB18070CDB199D4202D980256D02C7
:1074300052191D0C00041B04000C52191B18964213
:1074400035D300D1FCE001231943049E994FF5196F
:10745000002D00DCA1E0480709D00F230B40042BCE
:1074600005D00B1D8B42894149428B44191C5A4659
:10747000D20107D5904B5C46049E80271C40FF003C
:10748000A346F5198D4B9D427ADD039C01222240D3
:1074900000248B4DA146BDE68024240347462742A5
:1074A0004CD13C432403240B009A854DB2E6361997
:1074B000481EB4425ED9011C9642C4D1009E9E4231
:1074C000C1D1C2E7031C283B311C99408B460021E7
:1074D00084E6301C01F088F820306EE6283B211C41
:1074E00099400022884691464DE6201C01F07CF828
:1074F000203037E60021B14500D33DE7009F5A46D2
:10750000B944B945BF417F423F19FB18013A9C423B
:107510001ED2984200D97EE000D1B5E0191A9346F8
:107520002AE7894500D8ADE64846464642467708F0
:10753000D3074608C0071E438146AAE658462042A4
:1075400012D1044324032A1C240B89465C4D61E6B6
:10755000A342E3D1009F4F45DBD9211A93460BE7A5
:10756000171CDDE69B46BCE63C432403240B009A33
:10757000534D4FE6B24259D800D18AE0011C62E770
:107580005F46C9087B07039E0B437C026D05012201
:107590009946240B6D0D32403CE64A4B049FDB1BA1
:1075A000382B10DD039C0122224000240025A14637
:1075B00030E60121494248E7029304E71F1C21E716
:1075C000019C039441E71F2B40DC3F48049F0C1CA7
:1075D0003A1858469140DC40904020430A1C511E06
:1075E0008A41011C11435A46DA40131C480709D04E
:1075F0000F220A40042A05D00A1D8A4289414942C5
:107600005B18111C1A0234D5039C0122224000246D
:107610000125A146FEE5009F02214942B9448B4461
:10762000B945894149420919CB18A4E6009D881E35
:107630006900A942AD416D422C19361900913AE713
:10764000002B00D033E70024009437E71F4A049C46
:107650005D46121BD5402A1C202B1FD01C4E5F46B6
:10766000A3199F403B1C19434B1E99411143002312
:10767000BCE75A07C9080A43039F91465B020122EF
:107680001C0B3A400025C5E54E45C4D89346002161
:1076900072E6009F9F42C9D3011C0FE70023E2E777
:1076A000802424035F463C432403240B019A89462B
:1076B000034DAFE5FF030000FFFFFFFEFE070000E4
:1076C000FF07000002FCFFFF1E040000E2FBFFFFBB
:1076D0003E040000F0B5564644465F464D46F0B4C1
:1076E0001F1C0B031B0B9A464B0087B0041C8046E3
:1076F0005B0DC80F161C02938146002B68D0694BA6
:107700000299994232D08022534652031A43D20042
:10771000630F1A439246644AE0008918804602913A
:10772000002400253B031B0B9B467800FB0F321CFB
:10773000400D039300D175E05A4B984269D08022E6
:10774000594652030A43730FD2001A43564B9346CD
:10775000C018F200002303994E4671401C430F2CC1
:1077600000D9ABE0514EA4003459A74653461C4300
:1077700000D087E00025AA46A84608240225D1E7C4
:107780004946022D6CD0032D00D119E2012D00D005
:107790005AE10D40EDB20024A9460023A046002086
:1077A000002125030A0D1C052D0B1205404B2A4311
:1077B000134023435B004C465B08E207191C40461C
:1077C000114307B03CBC90469946A246AB46F0BD7B
:1077D0005346234350D05346002B00D186E15046F8
:1077E00000F002FF031E272B00DD78E128210D1A8F
:1077F000211C083B5246E9409A400D1C1543221CAF
:107800009A40AA4690462B4B00241B1A029300254F
:1078100088E75B461E430323002E9CD1B34600221B
:10782000022398E75B46334321D05846002800D115
:1078300050E100F0D9FE272800DD44E128210F1A8D
:10784000021C311C083A5B46F94093400F1C1F4351
:10785000331C9340BB461A1C164B181A00237AE7B8
:1078600001230B4000249946A0460E4B97E70027C2
:10787000BB46002201236EE7002104248A46884685
:1078800001254FE70C2403254CE701235B4200252B
:107890009846A946084C034B81E7DA46904603997F
:1078A0001D1C6EE7FF07000001FCFFFFD4B30200C0
:1078B000FFFF0F800DFCFFFFFFFF0F00029F160C64
:1078C000381804904046070C0004000C1204120CF7
:1078D000031C5343041C3D1C7443554398463B1CF6
:1078E00073436419A44644460293230C63449D42A7
:1078F00004D9029D802464022D1902951D0C039564
:1079000045462C041B04240C1C1905945C46230CCE
:10791000051C58432404240C8446381C60436543EA
:107920005F438146CC44280C6044BB46814502D964
:1079300080277F02BB442D04070C2D0C0004401946
:107940005546BC462F04E3448446280C3D0C2F1CAE
:107950005743B8462F1C77434243B94647463F0C2E
:107960009144BA46D14446434A4502D98022520244
:10797000B6184F463A0CB6183A0447463F043F0C37
:10798000B8462F1C67435D43444358436519019033
:10799000380C2D184244B846AC4204D901988023D3
:1079A0005B02C0180190039C029F201C6044C01918
:1079B0006045A44147466442A4462B043C049946D2
:1079C000240C4C44A046D8448018C246E24490425D
:1079D0009241574652429146F219E245BF417F42D9
:1079E0004B46BC46D845BF41D4187F4263461F432F
:1079F0002D0C7F19B24292414C45AD4152426D422D
:107A00001543019E7D19AB19E20D5B02059F1343DF
:107A100042023A439A46531E9A41C30D101C184322
:107A20006402204380465046C0010DD545460122E0
:107A30005646049C6B082A401A43F30701341A4344
:107A4000760804949046B246049E634FF319002BC7
:107A500061DD404640070BD00F2244462240042AF5
:107A600006D042460432424580414042824490461C
:107A70005546ED0107D5594B5646049F80201E40C0
:107A8000C000B2463B18564A934200DDE8E6444641
:107A90005546E2086807104301226C025B050A4064
:107AA0008046240B5B0D914679E6DA4690461D1C14
:107AB00067E680242403574627421CD13C43240315
:107AC000240B484B6BE6031C283B311C99408B462A
:107AD0000022C1E6301C00F087FD2030ABE6283BD9
:107AE000211C994000228A4690468CE6201C00F01A
:107AF0007BFD203076E65846204207D104430399A7
:107B00002403240B89469046364B48E63C43240325
:107B1000240B344B43E6344B049E9B1B382B06DD71
:107B200001230B4000249946A046002337E61F2B73
:107B300025DC049C2D4D464660195246444686403D
:107B4000DC4082405746301C2243DF40441EA041A7
:107B500002433B1C540709D00F201040042805D0D5
:107B6000101D9042924152429B18021C1D021AD5D0
:107B700001230B4000249946A04601230FE61C4830
:107B8000049C5546001BC540281C202B16D0194EBE
:107B90005746A21997403A1C43461A43531E9A412E
:107BA00002430023D6E758075B02D2081C0B0123CF
:107BB0000B401043994680460023F0E50022EBE796
:107BC0008024240350460123044319402403240B3A
:107BD0008946044BE3E5C046FF030000FFFFFFFEBC
:107BE000FE070000FF07000002FCFFFF1E0400006C
:107BF000E2FBFFFF3E040000F8B55F4656464446F0
:107C00004D46F0B40C034D00CF0F610A440F2143E1
:107C1000C4001803DE0F8046B44646465800760A74
:107C2000530F3343D600D14A6D0DBA46400DB346CB
:107C3000904200D1F5E062460126724094466745C5
:107C400000D1ABE02F1A002F00DC11E100283ED15B
:107C50005846184300D0F1E0600700D197E00F23A9
:107C60002340042B00D122E1221DA242A441644200
:107C7000802309191B04012750460B400740141CA0
:107C8000002B00D179E0B94B01359D4200D10BE1C9
:107C9000B74BE40819404807490204430B0B002086
:107CA00000211B031A0B0B0D6D051B0513436A08FE
:107CB000B04DFF071D4015436D006D08291C394369
:107CC000201C3CBC90469946A246AB46F8BDA7484E
:107CD0008542C1D0802000040343382F00DDFDE041
:107CE0001F2F00DD31E12020C01B1A1C5E468240A0
:107CF000FE40324394465A468240101C421E904138
:107D0000FB40624602431F1CA21A9442A4416442F3
:107D1000C91B091B141C0A029ED549024F0A002FD9
:107D200000D1D6E0381C00F05FFC021C083A1F2A84
:107D300000DDC3E02821231C091A9740CB401F43D4
:107D40009440954200DDC0E0551B691C1F2900DDF1
:107D5000EAE01F22551B3B1C221CAB40CA40AC4032
:107D6000651EAC411343CF401C43391C002573E70B
:107D7000082481497D4D002764427C4B4807E40874
:107D80000443C9089D4250D009030B0B87E78023A9
:107D90001B04012752460B40174071E72A1A9446EC
:107DA000002A00DCA1E0002854D07048854200D1B0
:107DB00052E78020000403436046382800DD10E1CC
:107DC0001F2800DD59E162462020801A1E1C8640D3
:107DD000B1465E46D6404A4632435E4686409046AD
:107DE000301C421E9041424602436046C340121975
:107DF000A242A441644259180919141C080200D473
:107E00002AE75A4B01359D4200D133E1584B6008B7
:107E10001940012323401C1C0443CB071C43490881
:107E20001AE71E4300D00AE705E7231C0B433BD0AB
:107E300080231B030B431B031B0B30E7013F002F69
:107E40006DD15E46A21B9442A4416442C91A091B2B
:107E5000141C60E75846184300D1FDE6012676421F
:107E6000B4446046002800D0D2E05E463219BFE735
:107E7000002F00D082E0681C4005400D012800DC86
:107E8000EAE05A46A21A9442BF41C81A7F42C71B71
:107E90003E0200D49AE05846041BA3459241591A69
:107EA00052428F1AE2463AE700230024F7E6802385
:107EB0001B04012756460B403740E1E6271C2838B3
:107EC00087400024954200DC3EE72949AD1A39403D
:107ED000C2E6201C00F088FB203026E75A461A43F1
:107EE000531E9A41D2B200270EE7002A00D0E0E0EC
:107EF000681C4605760D012E00DC92E01B4DA84261
:107F000000D1F7E05E463219A242A44164425918FA
:107F10000919CC07520814434908051C9CE613486C
:107F2000854200D0D9E697E62B1C1F3B3E1CDE4065
:107F3000331C202971D03F22551BAF403C43601EAB
:107F400084411C430021002586E6381C20381E1C75
:107F5000C640301C202F62D04022D71BBB405A465F
:107F60001A43531E9A4102430027CDE6FF07000043
:107F7000FFFF7FFFFFFF0F80FFFF7F00002D37D047
:107F8000B64DA84200D18FE080252D047F422943C1
:107F9000382F00DDA8E01F2F00DD24E12025ED1B98
:107FA0000E1CAE40B046261CFE404246AC40164376
:107FB000651EAC413443F9405A46141BA345924117
:107FC0005B1A5242991A051CE246A4E6131C3B4375
:107FD000141C002B00D0A2E600270021002400255D
:107FE000CBE65A461A43531E9A41D2B20023FEE60C
:107FF0000D1C254358D0FF43002F51D15A46141B66
:10800000A3459241591A5242891A051CE24682E65A
:108010009248854200D0CFE61EE600278EE7002377
:108020009DE7081C2043002D00D0C2E0002800D1AD
:10803000EFE05846184300D10EE658460219A24216
:10804000A441644259180919141C0A0200D403E619
:10805000834B01251940FFE5081C2043002D38D132
:1080600000286FD15946194303D0191C5C46E246DB
:10807000F2E50027002100247FE6604620381A1C24
:10808000C2406646101C202E00D1AAE04022921B5E
:1080900093405A461A43531E9A4102430023A6E6D0
:1080A0006E4DA84200D073E7191C5C46051CE246E1
:1080B000D2E5002D22D10D1C254376D0D543002DCD
:1080C00070D15C445C459241591852428918051C94
:1080D00094E600284CD15946194300D148E6191CB2
:1080E0005C46E2465D4DB7E50C43611E8C41E4B24F
:1080F000002161E7051C002100243EE6574DA842FF
:1081000053D05542802216043143382D7BDC1F2D7D
:1081100000DD8CE02022561B0A1CB446B240261C0F
:10812000EE403243904662469440661EB441424659
:108130001443E9405C445C459241CB185242991883
:10814000051C5BE65846184300D185E55E46A71B33
:10815000BC429241C81A5242801A060260D5584663
:10816000041BA3459241591A5242891AE24673E50B
:108170005846184333D04807E40804438020C90810
:108180000003014208D0DD08054205D15946CA085E
:108190005C071443291CE246630FC9001943E4003D
:1081A0002E4D59E52D4A9042AFD1191C5C46051C55
:1081B00052E5002830D05846184310D08025480793
:1081C000E408C9082D0304432942E5D0D808284211
:1081D000E2D15D46EA085C071443011CDCE71F4D51
:1081E0003AE5002355E73D1C203D0E1CEE40351CB2
:1081F000202F2ED04026F71BB9400C43611E8C4126
:108200002C430021D8E60C43611E8C41E4B20021CE
:1082100090E7191C5C461FE5191C5C460F4D1BE5D9
:10822000031C3B4300D124E7011C3C1C14E5202621
:10823000764276190A1CF2409046202D0BD040263B
:10824000751BA9400C43611E8C4145462C430021FF
:1082500070E70021D1E70021F4E7C046FF070000E6
:10826000FFFF7FFF70B50B1C124C09030E0B59006A
:10827000021C490DDD0F0020A14211DD0E48814294
:108280000FDC8020400306430C48401A1F280BDDFA
:108290000B4A521AD640321C5042002D00D1101CFD
:1082A00070BD084BE818FBE7074BC240C9188E4069
:1082B0003243F1E7FE0300001D0400003304000018
:1082C00013040000FFFFFF7FEDFBFFFFF8B5041E66
:1082D00031D0C70F00D04442201C00F085F9184D62
:1082E0002D1A0A2819DD0B38844024036D05240B50
:1082F0006D0D3A1C0026002000210B0D2403240BD9
:108300001B0523430F4C2D051C402C4364006408BF
:10831000D307211C301C1943F8BD061C1536231C3D
:10832000B3401E1C0B23181AC44024036D05240BF4
:108330006D0D3A1CDFE70022002500240026DAE755
:108340001E040000FFFF0F8010B5041E28D000F0AF
:108350004BF9154A121A0A2815DD0B3884402403FC
:108360005205240B520D0023002000212403181C69
:108370000B0D240B1B0523430C4C12051C4014430E
:108380006400610810BD031C1533211C99400B1CAF
:108390000B21081AC44024035205240B520DE3E7B5
:1083A000002200240023DFE71E040000FFFF0F80EF
:1083B00043001B0E5A1C4102D2B270B54C0AC50FC5
:1083C000012A17DDE02292006407090B98180022A9
:1083D00000231E0D221C34050C431B494005400898
:1083E0002140014349004908ED070B1C2B43101C99
:1083F000191C70BD002B15D1002C1CD0201C00F0C6
:10840000F3F80A281ADC0B21091A231CCB40191C8B
:10841000031C15339C400D4B0903181A4005090B2A
:10842000400DD4E7002C03D06407090B0848CEE7C1
:1084300007480021CBE700200021C8E7011C0B39C9
:108440008C40211C0024E6E7FFFF0F808903000019
:10845000FF070000F0B54B000D03420F5B0D6D0AE6
:1084600015435A1C5205CC0FC600520D012A27DDB8
:10847000394FDA19FE2A1ADC002A35DD8001ED00B9
:10848000431E98412843760F3043430704D00F23FF
:108490000340042B00D004308021C904014027D0C0
:1084A0000132FF2A1DD083015B0AD1B201E0FF2116
:1084B00000235802C905400AE40708432043F0BDE1
:1084C000002B06D1354311D10021002043025B0A65
:1084D000EFE72E43EBD08020ED0080042843FF22FD
:1084E000D3E7FF210023E4E717320DDA052000224D
:1084F000C008D1B2FF2AE9D10028D9D08023DB03FC
:1085000003435B025B0AD4E780221449120415433B
:10851000C91A1F290DDC124A371C9B18281C9F40C2
:1085200098403B1C5A1E93411843CE4030430022D2
:10853000ABE70C4F2A1CFF1AFA40171C202909D060
:10854000094A98188540281C3043461EB0413843DC
:1085500000229AE70020F7E780FCFFFF9E0300005F
:1085600082FCFFFF7E030000A2FCFFFF8446101C7C
:1085700062468C46191C634600E0C0461FB500F0F9
:10858000CFFC002801D40021C8421FBD10B500F067
:1085900003FC4042013010BD10B500F0C1FC0028C2
:1085A00001DB002010BD012010BDC04610B500F059
:1085B000B7FC002801DD002010BD012010BDC04621
:1085C00010B500F033FC002801DC002010BD0120B4
:1085D00010BDC04610B500F029FC002801DA0020CB
:1085E00010BD012010BDC0461C2101231B04984270
:1085F00001D3000C10391B0A984201D3000A083934
:108600001B09984201D30009043902A2105C4018EA
:108610007047C0460403020201010101000000008E
:10862000000000009C460304F0B51B0C17043F0C2F
:10863000150C1E1C041C000C7E436B434743454332
:10864000FB18300C1818874202D980235B02ED1802
:10865000030CED1863465C434A433604360CA118FC
:10866000000480194919F0BDF0B544465F465646EE
:108670004D46F0B41C1C85B0002900DAD9E00F1C6F
:108680000021061C8A46101C191C002C00DAC7E0C9
:108690000196009089468046002950D1B84262D99F
:1086A000FFF7A2FF002809D020234546311C1B1AE2
:1086B00085408740D940A8460F4386404246140C67
:1086C00013041B0C211C381C9B46FDF785F95B46E7
:1086D0004343051C211C381C9946FDF7C1F9330C96
:1086E00008041843814509D940446B1E804500D9D0
:1086F00077E1814500D874E1023D40444946411A82
:108700008946081C211CFDF767F95A464243071C9D
:10871000211C48469346FDF7A3F936040904360C9C
:108720000E43B34507D946447B1EB04502D8023FED
:10873000B34500D81F1C2D042F43002403E0B94289
:1087400060D9002400275246381C211C002A03D07F
:108750003B1C00215842A14105B03CBC90469946C3
:10876000A246AB46F0BD002804D101200021FDF750
:1087700033F980464046FFF737FF002860D1414675
:1087800044460B043C1B1B0CA3460D0C0093012418
:10879000291C5846FDF720F9009F81464743291CB4
:1087A0005846FDF75DF9330C090419438F4208D987
:1087B0004B464144013B884502D88F4200D925E110
:1087C0009946C91B8B46081C291CFDF705F9009B1F
:1087D000291C4343071C58460093FDF741F9360412
:1087E000009D0904360C0E43B54207D946447B1E52
:1087F000B04502D8023FB54200D81F1C49460B04C1
:108800001F43A0E7081CFFF7EFFE041E70D1B94517
:1088100003D3009C019DAC4293D80024012792E72A
:108820005246D243031C0C1C924600215842A141DF
:108830002EE7002746428F41012149428A4622E71E
:1088400020231B1A4246351C82403C1CDD40DC4084
:1088500087402B1C150C3B43291C8640201C009391
:1088600017049046FDF7B8F83F0C011C7943814688
:108870008B46201C291CFDF7F3F8009C0904230CEF
:1088800019438B450CD94B464144013B884500D9DF
:10889000BAE08B4500D8B7E00222524291444144ED
:1088A0005C460C1B201C291C0194FDF795F8391C13
:1088B0004143041C8B460198291CFDF7D1F8009A0E
:1088C000090413041B0C19438B4509D94144631E49
:1088D000884500D994E08B4500D891E0023C4144A2
:1088E0005B46CB1A49469B460B041C4300974FE757
:1088F000009D20231B1A4A4600998240DD40154303
:1089000081403A1CDA400091311C9046D9403A1C13
:1089100082400B1C134301932F0C2B041B0C391C9E
:1089200040460293FDF758F8029A81464243391CAB
:1089300040469346FDF794F8019A0904130C194335
:108940008B450AD94B464919013B8D425AD88B4574
:1089500058D902235B42994449195A468A1A101C75
:10896000391C0392FDF738F8029B80464343391CBB
:1089700003989B46FDF774F8019A090413041B0C35
:1089800019438B450AD943464919013B8D4235D8D5
:108990008B4533D902235B42984449195D464D1BF0
:1089A000AB464946009D0F04424617432A04120C69
:1089B0003B042D0C1B0C380C111C594342436B43D8
:1089C0006843D3180D0C5B198C469A4202D9802259
:1089D000520280181D0C401983450CD303D000248B
:1089E000B1E61D1C8AE665462A041B04120C9B187E
:1089F000A6409E42F3D2013F0024A4E69846CDE76C
:108A00001C1C6DE79946A8E7994649E702225242A5
:108A100091444144D5E6C046F0B55F4656464D46C2
:108A20004446F0B40D1C85B0061C92469846029050
:108A3000019103921F1C141C8346A946002B52D19E
:108A4000AA426BD9101CFFF7CFFD00280AD02023C3
:108A50001B1A311CD94085400B1C2B438640844097
:108A60009946B346250C23041B0C291C48469846FE
:108A7000FCF7B2FF4646071C4643291C4846FCF754
:108A8000EFFF5A460904130C19438E4209D90919FC
:108A90007B1E8C4200D959E18E4200D856E1023F3C
:108AA0000919891B8946081C291CFCF795FF4346B8
:108AB0004343061C291C48469846FCF7D1FF5A46FA
:108AC000130409041B0C1943884508D90919731E9E
:108AD0008C4200D938E1023E884500D834E13804A0
:108AE0003043002712E0019A93420DD8181CFFF77B
:108AF0007BFD041E66D1019B9F4200D221E1039FB2
:108B000002998F4200D81CE100270020391C05B0D3
:108B10003CBC90469946A246AB46F0BD002A04D123
:108B200001200021FCF758FF041C201CFFF75CFD0E
:108B3000002800D0B6E023042D1B1B0CA946260CF0
:108B400098460127311C4846FCF746FF4146414301
:108B5000051C8A464846311CFCF782FF5A46080429
:108B6000130C1843824507D900196B1E844202D8A2
:108B7000824500D90DE11D1C5346C31A181C311C37
:108B80009A46FCF729FF41464143814688465046B4
:108B9000311CFCF765FF5A46130409041B0C1943EA
:108BA00088450BD94B460919013B8C4200D9CFE0CF
:108BB000884500D8CCE002235B429944280449460A
:108BC0000843A3E720231B1A424657468240DF4052
:108BD0001743524682400192321CDA40291CD94088
:108BE0008540131C2B4302933D0C3B041B0C884611
:108BF000081C291C9A46FCF7EFFE53464343814666
:108C0000291C40469B46FCF72BFF029A0904130CD3
:108C100019438B4506D94B46C919013B8F4200D8F1
:108C2000ABE099465A468A1A101C291C9346FCF759
:108C3000D3FE53464343291C804658469A46FCF7C8
:108C40000FFF029A090415042D0C29438A4506D901
:108C50004346C919013B8F4200D886E098465746E3
:108C6000CF1BBA464946019F0804424610433D04C3
:108C70002D0C03043F0C1B0C020C291C59435543BB
:108C80007B437A43EB180F0CDB198C469D4202D9CB
:108C900080277F02D2191D0C5219924562D359D0F8
:108CA000002733E720231B1A311C2F1CD940DF403B
:108CB00085400B1C84402B4386400193B34623041C
:108CC000260C1B0C381C311C9846FCF785FE4246CE
:108CD0004243051C311C381C9146FCF7C1FE019F24
:108CE00009043B0C1943894507D909196B1E8C42AD
:108CF0004DD889454BD9023D09194A468A1A101C9C
:108D0000311C9246FCF768FE43464343071C311C66
:108D100050469946FCF7A4FE019A090413041B0C63
:108D20001943894507D909197B1E8C422DD88945DD
:108D30002BD9023F09194B46CB1A2D0499462F43D4
:108D400000E700270120E1E61E1CC8E61F1CA8E67C
:108D5000994633E761460A041B04120C9B18A6408F
:108D60009E429DD201380027D0E68A4500D875E79B
:108D700002235B429844C91971E78B4500D850E73C
:108D800002235B429944C9194CE71F1CD3E71D1C01
:108D9000B3E7023D0019EFE6F0B55F4656464D4693
:108DA0004446F0B40D1C041C8046E80F81461803AD
:108DB0000F03000B3F0B83B084461B48009749000C
:108DC0005E00DF0F490D9246760DBB4681420CD006
:108DD0001548864210D00120B14215D003B03CBCEA
:108DE00090469946A246AB46F0BD009F012027431E
:108DF000F4D10D488642EED1604602430120002A9C
:108E0000ECD10120B142E9D1009B6345E6D1D045C8
:108E1000E4D1D94506D00029E0D11C43201C441ED2
:108E2000A041DBE70020D9E7FF070000F0B55F466F
:108E300056464D464446F0B4CD0FDE0FAC461D03FA
:108E40002D0BB146354E0F034C00AB465D008046FE
:108E50003F0B640D92466D0DB44231D02F4EB5429A
:108E600034D0002C0ED1384341424141081C002D22
:108E70000BD0002919D1CC452CD06646002E17D135
:108E8000012017E0002DF6D1281C59460A43534211
:108E90005341002806D1002BEDD065460120002D5E
:108EA00008D005E00020002B04D14B46002BE7D171
:108EB000012040423CBC90469946A246AB46F0BDDC
:108EC0003E1C0643CAD002204042F3E75E461643EA
:108ED000C7D0F8E7AC4205DC09DA6346002BE7D0DF
:108EE0000120E7E761460029E2D10120E2E75F4582
:108EF00008D80CD000205F45DCD26646002ED7D0C3
:108F00000120D7E76546002DD2D10120D2E7D04518
:108F1000F8D80020D045F0D3CCE7C046FF070000CA
:108F2000F0B556464D4644465F46F0B40D1C83B03E
:108F3000041C0190E80F814618030F03000B3F0B40
:108F400084463848009749005E00DF0F490D92467D
:108F5000760DB846814233D03248864235D000295A
:108F600017D0002E1ED1341C67463A43534253415A
:108F7000002C1ED00020002B04D14046002816D122
:108F80000120404203B03CBC90469946A246AB4605
:108F9000F0BD0098044360426041041C002EE3D001
:108FA0000028EAD1C14515D04F46002FE8D1012055
:108FB000E8E7002BF6D04B460120002BE2D0DFE79C
:108FC000009F02202743DDD1C6E7674602201743F2
:108FD000D8D1C4E7B14204DD48460028D0D10120F1
:108FE000D0E7B14204DA4B46002BC9D00120C9E7D3
:108FF000009F674509D80DD0009F00206745C1D26A
:109000004F46002FBCD00120BCE74B46002BB7D108
:109010000120B7E701985045F7D8019B0020534540
:10902000EED3AFE7FF07000008B50A1C0349031C95
:109030000868191C00F00DF808BDC0466024002027
:1090400010B50023934203D0CC5CC4540133F9E73C
:1090500010BD38B5151C4D43291C00F051F8041EF5
:1090600003D000212A1CF7F7A3F8201C38BD00000C
:1090700030B5002940D004390B68002B00DAC9183C
:109080001E4A1368141C002B02D14B60116033E0A0
:1090900099420FD208680A189A4205D1136852689B
:1090A000C01808604A6000E04B60216024E08A42FA
:1090B00003D8131C5A68002AF9D11D685C198C4228
:1090C0000BD10968691858181960904214D11468B6
:1090D0005268091919605A600EE08C4202D90C23BB
:1090E000036009E008680C18944203D114685268C0
:1090F000001908604A60596030BDC046502F0020FA
:1091000070B50323CD1C9D430835061C0C2D01D2E0
:109110000C2501E0002D3FDB8D423DD3204B1C6828
:109120001A1C211C002913D00868431B0DD40B2BDB
:1091300002D90B60CC181EE08C4202D16368136028
:109140001AE0486860600C1C16E00C1C4968E9E7EE
:10915000144C2068002803D1301C00F025F8206052
:10916000301C291C00F020F8431C15D0C41C03231C
:109170009C4384420AD12560201C0B300722231D0A
:109180009043C31A0BD05A42E25008E0211A301C17
:1091900000F00AF80130EED10C233360002070BDDE
:1091A000502F00204C2F002038B5074C0023051C01
:1091B000081C236000F076FB431C03D12368002BBE
:1091C00000D02B6038BDC046682F00200EB400B51B
:1091D0009CB01DAB04CB822202A992008A810A4A6C
:1091E00002908A604A6101225242CA81074A08619C
:1091F00010681D9A019300F087F8029A00231370FB
:109200001CB008BC03B01847FFFFFF7F602400209C
:109210000023C25C0133002AFBD1581E704730B5D1
:10922000031C002A07D00C7801335D1E013A2C7014
:109230000131002CF5D19A18934203D00021197006
:109240000133F9E730BD0000F0B58D6885B0071C2B
:109250000C1C03920193AB4245D390228B89D20020
:1092600013423DD062690326564309692068F20F14
:10927000401A96190290021C0198013212187610B9
:10928000964200D2161C381C5A050FD5311CFFF728
:1092900037FF051E13D0029A2169FFF7D1FEA2897C
:1092A000184B134080221343A38111E0321C00F0BD
:1092B000C9FA051E0CD1381C2169FFF7D9FE0C2311
:1092C0003B60A389402213430120A381404217E061
:1092D000029B2561ED1825606661019DF61AA66066
:1092E0000198A84200D2019D2A1C2068039900F031
:1092F00090FAA2680020531BA36023685D192560C3
:1093000005B0F0BD7FFBFFFFF0B59FB005938B89E3
:1093100003900E1C171C19060FD53269002A0CD1B8
:109320004021FFF7EDFE30603061002803D1039942
:109330000C230B60C9E04023736106AD00236B6111
:1093400020236B763023AB763C1C2378002B03D193
:10935000E21B029211D003E0252BF9D00134F4E78F
:109360000398311C3A1C029BFFF76EFF013000D1BD
:10937000A6E06969029A8B186B612378002B00D1F3
:109380009EE0012252426A606A4600235B32013449
:109390002B60EB60AB601370AB654E4F2178381CCF
:1093A000052200F02BFA002807D0C71B2B680120EC
:1093B000B840184328600134EFE72B68D90603D57D
:1093C0006A4620215B3211701A0703D56A462B21A9
:1093D0005B32117022782A2A01D0099B0EE0059A8F
:1093E000111D12680591002A01DB099204E0524226
:1093F000EA60022213432B60013409E02278303AFC
:10940000092A04D80A214B4301349B18F6E7099333
:1094100023782E2B18D163782A2B09D1059B02348F
:109420001A1D1B680592002B0DDA01235B420AE02E
:10943000013400232278303A092A04D80A214B4308
:1094400001349B18F6E70793234F2178381C032239
:1094500000F0D4F9002806D0C71B2B684020B84084
:1094600018432860013421781C480622671C29769D
:1094700000F0C4F9002812D0194B002B06D1059B2F
:109480000722073393430833059314E005AB009399
:109490000398291C321C134B00E000BF07E005AB0A
:1094A00000930398291C321C0E4B00F091F8049095
:1094B0000499013104D06A69049953186B6143E738
:1094C000B3895A0601D40B9801E0012040421FB035
:1094D000F0BDC04614B402001AB402001EB402006B
:1094E0000000000049920200F7B5151C01930A69BB
:1094F0008B68061C0C1C934200DA131C221C2B6088
:1095000043321278002A01D001332B602068800694
:1095100002D52B6802332B60216806270F401FD02D
:10952000231C43331B785A1E9341226892061FD591
:10953000E11840313020C870211C5A1C453109788F
:10954000A21840320233D17012E0221C301C019963
:1095500019320123089FB847013011D0009F01370D
:109560000097E0682968009F431A9F42EDDBD7E728
:10957000221C301C01994332089FB847013002D1A8
:109580000120404223E0206806212B68E268014068
:109590000025042903D1D51AEB43DB171D40A2682F
:1095A00023699A4201DDD31AED1800270097009F26
:1095B000AF420BDA221C301C01991A320123089F9A
:1095C000B8470130DCD0009F0137EFE70020FEBD37
:1095D000F0B58BB007930D1C0B7E433506920590BA
:1095E0000C1C109A04956E2B00D1A7E011D8632BA8
:1095F00022D009D8002B00D1B0E0582B00D0C0E019
:1096000045310B707B4D4EE0642B1CD0692B1AD07A
:10961000B7E0732B00D1A5E009D86F2B29D0702BB0
:1096200000D0AEE00E68202333430B6036E0752B8C
:109630001FD0782B32D0A4E013680D1C191D4235C1
:1096400011601B689FE0216813680E0603D5191D81
:1096500011601E6805E04806F9D5191D116000214A
:109660005E5E644B002E3BDA049D2D2276422A700A
:1096700036E0216813680E0603D5191D11601E68B7
:1096800004E04806F9D5191D1E881160594B227E49
:10969000039308276F2A1ED00A271CE0231C782179
:1096A0004533554D197011682368081D03951060E6
:1096B0001E0601D50E6802E05806FBD50E88D907B4
:1096C00002D52022134323601027002E03D12268E5
:1096D00020239A432260231C002243331A7001E0A6
:1096E00003930A276368A360002B03DB2568042229
:1096F00095432560002E02D1049D002B0ED0049DC1
:10970000301C391CFCF7ACF90398013D435C301C5C
:109710002B70391CFCF760F9061EF1D1082F09D116
:109720002168C90706D5626823699A4202DC013DB7
:1097300030232B70049E731B23612AE00868136892
:109740004969050604D5181D10601B68196005E0FD
:109750004606F8D5181D10601B6819800023236188
:10976000049D16E01368191D11601D68281CFFF781
:109770004FFD63682061984200D9236120696060D1
:1097800004E0251C42352B7001232361049E002335
:109790003370079E05980096211C09AA069BFFF7C7
:1097A000A3FE013002D10120404221E02A1C05988D
:1097B00006992369079DA8470130F4D02668B607AB
:1097C00005D4099BE068984212DA181C10E00025C5
:1097D000E0680999431A9D42F3DA221C059806991C
:1097E00019320123079EB0470130DCD00135EFE785
:1097F0000BB0F0BD25B4020036B40200C9B2821825
:10980000904204D003788B4202D00130F8E7002068
:10981000704770B5814201D300230CE08C18A04240
:10982000FAD28518131C013B0BD351426618F65C23
:109830006918CE54F7E7934203D0CC5CC45401338B
:10984000F9E770BDF8B5061C0C1C151C002904D1E5
:10985000111CFFF755FC041C18E0002A03D1FFF788
:1098600007FC2C1C12E000F013F8A8420ED2301CAA
:10987000291CFFF745FC071E07D0211C2A1CFFF7F7
:10988000DFFB301C211CFFF7F3FB3C1C201CF8BD48
:1098900004390B68181F002B02DAC8581B18181F50
:1098A00070470000094A1368002B0CD0181869464D
:1098B000884202D81060181C7047054B0C2201200A
:1098C0001A604042F8E7034B1360EFE7542F002083
:1098D000682F0020702F0020F0B5474680B4284A3A
:1098E0004F007F0DBE180D1C8C46132E1ADC002E67
:1098F0003ADB244F021C37413B1C0B4003439C4680
:109900000B1C6146002908D080231B0333415E19DC
:10991000BE43B446002763463A1C101C191C04BC05
:109920009046F0BD332E0BDD0B1C8021021CC900BC
:109930008E42F2D1291CFDF781F8021C0B1CECE7CA
:10994000114A0126BB187642DE40021C0B1C06425F
:10995000E3D00E4BDF1B0123BB401F18B84201D9D7
:109960004B1C9C46B743D6E7CB0FDB079C46002732
:109970000136D0D1064B614619438C46CBE7C04631
:1099800001FCFFFFFFFF0F00EDFBFFFF32040000B3
:109990000000F03F00000000F0B5474680B48CB0F6
:1099A000141C1D1C061C0F1C00F016FA2C4A002368
:1099B000D356904600900191013305D0201C291CFC
:1099C00001F0DCF9002805D1009801990CB004BC25
:1099D0009046F0BD301C391C01F0D0F90028F3D0BE
:1099E000201C291C1D4B1C4AFEF7D0FD0028EBD083
:1099F000012302931B4B06940795039300230A93BC
:109A000043461C7804960597002C15D0134912483C
:109A1000021C0B1CFDF736FB08900991022C0DD19E
:109A200001F022FB212303600A9C002C0CD1089B2F
:109A3000099C00930194C7E70896099702A801F0D2
:109A4000CDF90028F0D1EBE701F00EFB0A9A026095
:109A5000EDE7C046C046C046000000000000000020
:109A6000AC24002048B40200F0B546464F46C0B4CE
:109A70008FB0161C1F1C0090019100F0FDFABC4A2B
:109A80000023D356041C0D1C904602940395013309
:109A900005D0301C391C01F071F9002806D102985C
:109AA00003990FB00CBC90469946F0BD00980199FF
:109AB00001F064F98146002831D1301C391CA14BDA
:109AC0009F4AFEF763FD0028E9D001230493A94BC8
:109AD00004AC63604B462362009A019BA260E36082
:109AE000994A9A4BA261E36142460023D35626610C
:109AF00067615A1C0ED0022B0CD0201C01F06EF9AD
:109B0000002800D17BE0236A002B03D001F0ACFADF
:109B1000236A0360A269E36902920393BFE7009896
:109B20000199884B864AFEF731FD002822D0301C6F
:109B3000391C844B824AFEF729FD051E2CD00123D7
:109B400004938C4B04AC636000232362009A019B56
:109B5000A260E3607B4B7A4AA261E3614246002344
:109B6000D35626616761002BC7D0774A774BA26135
:109B7000E361CFE7201C291C01F0F8F8814600289A
:109B800042D0201C291C6F4B6D4AFEF7FFFC0028B9
:109B90006CD10294039582E7301C391C01F0E6F881
:109BA000002800D17BE7301C391C664B644AFEF765
:109BB000F3FC002800D172E7012304936D4B04AC41
:109BC0006360009A019BA260E360434619782562B6
:109BD00026616761002900D17AE05D4A5D4BA26190
:109BE000E36102293CD101F03FFA21230360236A9B
:109BF000002B8FD001F038FA226A02608AE701F068
:109C000033FA212303607EE70098019901F0AEF852
:109C10000028B6D0301C391C01F0A8F80028B0D0BC
:109C2000201C291C01F0AAF804AC002855D10123FE
:109C30000493504B20626360009A019BA260E36032
:109C400043461D7826616761002D41D03D493C485F
:109C5000021C0B1CFDF716FAA061E161022DC2D0B7
:109C6000201C01F0BBF80028C1D1BCE70098019985
:109C700001F07CF802940395002800D10FE7301C16
:109C8000391C01F073F802940395002800D106E70F
:109C900004AC0423049326616761364B63600023A0
:109CA0002362009A019BA260E360264B244AA261D2
:109CB000E36142460023D356022B04D0201C01F05E
:109CC0008DF8002893D101F0CFF9222303608EE7AD
:109CD0001C4B1B4AA261E361C2E703230493254B9B
:109CE0002661676163604B462362009A019BA26014
:109CF000E36042460023D356002B3DD1164A174B52
:109D000000980199A261E3610E4B0D4AFEF744FCF5
:109D10000028CED0124A134B301C391CFDF7DAFC58
:109D2000061C0F1C01F064F8321C3B1CFEF72EFCD5
:109D30000028BED10C4A0D4BA261E361B9E7C046D1
:109D40000000000000000000000000000000F03FE4
:109D5000000000000000F0FF000000E0FFFFEF4700
:109D6000000000000000E03F000000E0FFFFEFC740
:109D7000AC24002050B40200104B0F4A0098019907
:109D8000A261E3610E4A0F4BFEF706FC002890D05B
:109D90000D4A0E4B301C391CFDF79CFC061C0F1C99
:109DA00001F026F8321C3B1CFEF7F0FB002800D027
:109DB0007FE7074A074B7AE7000000000000F07FCA
:109DC0000000000000000000000000000000E03F74
:109DD000000000000000F0FFF0B556464D46444636
:109DE0005F46F0B485B002900391029C5E00760855
:109DF0000194B446141C1D1C0092164330D0039FDE
:109E0000039EFF0FFF07B9467740B8468E4FB8450F
:109E100026DC56421643F60F67463E43B3468B4E4A
:109E2000B3451DD8E04506DC20DB019A009B9A4231
:109E30001CD300D1B4E0864B98451EDC4646002E6C
:109E400000D0BEE00198029B824A002819DD009FE5
:109E5000061C013A5B00002BFBDC0196009710E02A
:109E6000FDF738FC021C0B1CFDF70CF905B03CBCDF
:109E700090469946A246AB46F0BD4346764E1A152B
:109E80009219734B9C4511DC6746002F00D08FE080
:109E90000098231C6F4900280CDD019E071C013926
:109EA0005B00002BFBDC0196009703E063466A4EE3
:109EB00019158919694B9A4264DB47463B03802098
:109EC0001B0B40031843654B99424CDB2B03802549
:109ED0001B0B6D031D43019E009F521A002A15D0D3
:109EE000BE42A441431B64421B1B09D4F61B181C31
:109EF000304355D0F00F5B0018187600013AEDE7BB
:109F0000F40F400000197600013AE7E7BE429B419A
:109F1000451B5B4201960097ED1A00D580E0F61BC9
:109F20000196019B2B4373D0494A954208DC019E60
:109F3000F30F6D00ED18760001399542F8DD0196BA
:109F4000464B994259DA5B1A142B6BDC444C019E48
:109F50002F1C0919DE408F401D413E432B1C4946F2
:109F60001943301C82E75B1A1F2B3EDC3C4E6746D0
:109F70008D19261CEE40351C261C9F409E403D43FB
:109F80000096A8E79E1A1F2E27DC354F4046D319AE
:109F9000029FB040DF40029B3843B340019392E7F9
:109FA0004C46E30F2F4ADB00D318186859685DE769
:109FB000FB022A49019E009F01395B00002BFBDC5C
:109FC00071E7F302254A002B00DC5AE7019E009F4F
:109FD000013A5B00002BFBDC3FE72348029E801A1E
:109FE00086400023301C01936DE71F4D271C6D1A1E
:109FF000AF4000233D1C00936DE71C4F1C4A4846B0
:10A00000ED1905438B181B05291C194301982DE7F1
:10A010004E46F30F134ADB00D3181868596825E73A
:10A02000051C7EE71F2B08DC0D4A01988E18B540F1
:10A03000D8402E1C06434B4691E70B4E4B46711AF7
:10A040002E1C0E418BE7C046FFFFEF7F0000F07F24
:10A05000FFFF0F00EDFBFFFF01FCFFFF02FCFFFF16
:10A060001E04000058B40200E2FBFFFF0000F0FFF6
:10A07000FF03000000000000F0B55F4656464D4665
:10A080004446F0B499464B465C00934664088FB052
:10A090000D1C0F1C5A46211C0090061C8246029380
:10A0A0005846114337D069004908884668490495E5
:10A0B00088452BDC28D066498C4227DC00D180E023
:10A0C000002108910499002900DA7EE0002833D1AC
:10A0D0005F4B9C4200D196E05E4B9C426AD0029856
:10A0E0008023DB05984201D100F0E1FB5A4B029935
:10A0F000994221D1049A002A1EDB291C009800F005
:10A100004BFD061C0D1C08E0002ED4D0534A131C36
:10A11000434433430AD14F4D0026301C291C0FB055
:10A120003CBC90469946A246AB46F0BD4C4800F078
:10A1300057FE061C0D1CF0E70098291C00F012FECB
:10A14000534606908C46002B20D0FB0F013B049316
:10A15000049E089B33436AD0424B9C4200DC8DE056
:10A16000414B9C4201DC00F035FC404B984500DC43
:10A1700089E3029E002E00DC89E334493248021C48
:10A180000B1CFDF7A7FA061C0D1CC6E7404600286D
:10A1900004D0304BBA0092089A42D6D1029C002CCF
:10A1A00001DA00F0C4FB049E002E00DA73E3069E81
:10A1B0006546B2E7029C002C01DA00F076FC009EB6
:10A1C000ABE7002800D17BE7A0E729498C422BDCD4
:10A1D00026498C4200DC79E721158C4625498C45BF
:10A1E00001DC00F086FC244B61465B1A111CD9404F
:10A1F0000A1C9A40824200D068E701220A400223EA
:10A200009B1A089362E7154A131C4344334300D159
:10A2100081E7164B984500DC7FE3029C002C00DAB6
:10A2200035E35E464D4678E7022108914EE70098F7
:10A23000009A291C2B1CFDF7DFFC021C0B1CFCF7F1
:10A2400021FF061C0D1C68E79C7500883CE4377EE6
:10A250000000F07F0000F03F0000E03F000010C071
:10A260004CB402000000E0410000F043FFFFEF3F6C
:10A27000FFFF3F431304000033040000E24A0023C1
:10A28000904509DC0698C54BC34A6146FDF722FAA2
:10A290003523069088465B424046DC490215521839
:10A2A000D21892460303DA4DDA4A1B0B1D43934240
:10A2B00001DC00F0F6FBD84A934201DC00F036FCEA
:10A2C000D64B01229244ED1800240021069A2B1C43
:10A2D00006920793C900D24B8846434418685968D0
:10A2E0000A900B910A9A0B9B06980799FDF784FC3C
:10A2F0000A9A0B9B061C0F1C06980799FCF79EFBFD
:10A30000021C0B1CA648A749FCF7BCFE0C900D9143
:10A310000C9A0D9B301C391CFDF7DCF9029003915F
:10A320000B1C802189056D10802000220D43000345
:10A33000009201939C4A9D4B29180B190098019992
:10A34000141C1D1CFDF7C6F9021C0B1C301C391C0B
:10A35000FDF752FC0A9A0B9B061C0F1C201C291CA3
:10A36000FDF74AFC021C0B1C06980799FDF744FCFC
:10A37000021C0B1C00980199FDF7ACF9021C0B1C88
:10A38000301C391CFDF738FC0C9A0D9BFDF7A2F927
:10A390000690079102980399021C0B1CFDF79AF98D
:10A3A000041C0D1C221C2B1CFDF794F9804A814BC8
:10A3B000061C0F1C201C291CFDF78CF97E4A7F4BC4
:10A3C000FCF73CFB221C2B1CFDF784F97C4A7D4BDF
:10A3D000FCF734FB221C2B1CFDF77CF97A4A7B4BE3
:10A3E000FCF72CFB221C2B1CFDF774F9784A794BE7
:10A3F000FCF724FB221C2B1CFDF76CF9764A774BEB
:10A40000FCF71CFB021C0B1C301C391CFDF762F90D
:10A41000029A039B041C0D1C00980199FCF70EFB8B
:10A42000069A079BFDF756F9221C2B1CFCF706FB2E
:10A43000061C0F1C00980199021C0B1CFDF74AF921
:10A44000674A684B0A900B91FCF7F8FA321C3B1CE8
:10A45000FCF7F4FA00240D1C221C009801992B1C17
:10A46000FDF738F9221C2B1C0090019106980799E2
:10A47000FDF730F95A4A5B4B06900791201C291CC6
:10A48000FDF7BAFB0A9A0B9BFDF7B6FB021C0B1CEF
:10A49000301C391CFDF7B0FB029A039BFDF71AF93B
:10A4A000021C0B1C06980799FCF7C8FA061C0F1C27
:10A4B000321C3B1C00980199FCF7C0FA4A4A4B4BEE
:10A4C0000024201C0D1CFDF705F9494A494B069054
:10A4D0000791201C291CFDF7FDF8009A019B0290B2
:10A4E0000391201C291CFDF787FB021C0B1C301C50
:10A4F000391CFDF781FB404A404BFDF7EBF8021C8D
:10A500000B1C02980399FCF799FA464B43441A68CE
:10A510005B68FCF793FA061C50460F1CFDF7D6FE4D
:10A520000D1C4149041C41440A684B680698079970
:10A5300002920393321C3B1CFCF780FA029A039BA5
:10A54000FCF77CFA221C2B1CFCF778FA00220B1C6F
:10A5500000920193101C2B1C221CFDF74DFB029A4C
:10A56000039BFDF749FB069A079BFDF745FB021C81
:10A570000B1C301C391CFDF73FFB02900391089B1C
:10A58000049C013B234300D0C2E11D481D490490B7
:10A5900005914BE0C046C04600000000000040436B
:10A5A000000000000000F03F00000000000000007C
:10A5B000EF4E454A287ECA3F65DBC9934A86CD3FA8
:10A5C00001411DA96074D13F4D268F515555D53F8E
:10A5D000FFAB6FDBB66DDB3F033333333333E33F26
:10A5E0000000000000000840000000E009C7EE3F46
:10A5F000F5015B14E02F3EBEFD033ADC09C7EE3FD8
:10A60000000000000000F0BFFFFF0F0001FCFFFF93
:10A610000000F03F8E98030079B60B000000F0FFB9
:10A6200088B4020078B4020068B402000026321C2C
:10A630004B4658464946FDF7DFFA009A019BFDF765
:10A6400049F8029A039B041C0D1C58464946FDF725
:10A6500041F8021C0B1C201C291CFCF7EFF9009A86
:10A66000019B02900391301C4946FDF733F800909E
:10A670000191009A019B02980399FCF7DFF9CC4BFA
:10A68000041C0D1C0F1C8846994200DC19E1C94AC4
:10A690008B18034300D012E2AC4BAB4A02980399EB
:10A6A000FCF7CCF9009A019B08900991201C291C09
:10A6B000FDF7A2FA021C0B1C08980999FDF780FF10
:10A6C000A946002800D0FAE14A46BB4B8024111568
:10A6D0006403C918201C0841C11948009C4A9D4BBD
:10A6E0000B1C0903B54E090B400D0C43B4498519E9
:10A6F000B44E081A04412E414046B343A1460028F7
:10A7000000DA1EE200980199FDF776FA00900191B7
:10A71000009A019B02980399FCF790F94A461205AA
:10A7200090460024201C8C4A8C4B0D1C0F1CFCF7FF
:10A73000D1FF009A019B08900991201C291CFDF76C
:10A740005BFA021C0B1C02980399FDF755FA844A28
:10A75000844BFCF7BFFF844A844B261C0D1C041C51
:10A76000391C301CFCF7B6FF021C0B1C201C291CDA
:10A77000FCF764F9041C0D1C221C2B1C0898099979
:10A78000FCF75CF9089A099B061C0F1CFDF734FACC
:10A79000021C0B1C201C291CFDF72EFA321C0090F9
:10A7A00001913B1C301C391CFCF794FF704A714B23
:10A7B000041C0D1CFCF78EFF6F4A704BFDF71CFA52
:10A7C000221C2B1CFCF786FF6D4A6E4BFCF736F9FA
:10A7D000221C2B1CFCF77EFF6B4A6C4BFDF70CFA1E
:10A7E000221C2B1CFCF776FF694A6A4BFCF726F902
:10A7F000221C2B1CFCF76EFF021C0B1C301C391C8E
:10A80000FDF7FAF9041C0D1C221C2B1C301C391CF2
:10A81000FCF760FF604A614B02900391201C291CE9
:10A82000FDF7EAF9021C0B1C02980399FCF72AFCBD
:10A83000009A019B041C0D1C301C391CFCF74AFFBC
:10A84000009A019BFCF7FAF8021C0B1C201C291C27
:10A85000FDF7D2F9321C3B1CFDF7CEF90B1C021C94
:10A860004F485049FDF7C8F9464673181C15002C8F
:10A8700000DC60E1021C04980599FCF72BFF061C24
:10A880000D1CFFF74AFC029C002C00DA75E4002640
:10A890000025FFF742FC4C48089C031C434423431B
:10A8A00000D01AE106986146069A6346C3E4291C63
:10A8B0002B1C0098009AFCF70DFF061C0D1CFFF7DF
:10A8C0002CFC4B005B089946404B994500DC25E188
:10A8D0003F480B1823430DD1009A019B201CFDF724
:10A8E0008BF9021C0B1C02980399FDF75FFE0028F0
:10A8F00000D1E9E62C4A2D4B04980599FCF7EAFEB5
:10A90000294A2A4BFCF7E6FE061C0D1CFFF705FC46
:10A910002349244A0491059288E6029E002EB6DA65
:10A9200080200006051C5E464D44FFF7F6FB069AA4
:10A9300063461B481B49FCF7A5FB06908C46FFF7B6
:10A9400032FCC046C046C046FE822B654715973C88
:10A95000000000000000000000000000432EE63F61
:10A96000EF39FAFE422EE63F396CA80C615C20BE3E
:10A97000D0A4BE726937663EF16BD2C541BDBB3E05
:10A980002CDE25AF6A56113F93BDBE166CC1663FE3
:10A990003E5555555555C53F00000000000000408C
:10A9A000000000000000F03F59F3F8C21F6EA5013F
:10A9B000FFFF8F40000070BF02FCFFFF01FCFFFFA4
:10A9C00013040000FFFF0F00000010C0FFCB9040F9
:10A9D00000346F3F6C4B984500DC54E76B4B984557
:10A9E00001DDFFF7C6FB6146584B574A0698FDF755
:10A9F00003F9574A574B041C0D1CFCF76BFE564AD3
:10AA0000564B061C0F1C201C291CFCF763FE221C45
:10AA1000009001912B1C201C291CFCF75BFE504A66
:10AA2000504B02900391201C291CFCF753FE021C82
:10AA30000B1C4D484D49FDF7DFF8221C2B1CFCF781
:10AA400049FE021C0B1C4A484A49FDF7D5F8021C76
:10AA50000B1C02980399FCF73DFE474A474BFCF755
:10AA600039FE021C0B1C00980199FDF7C5F8041C67
:10AA70000D1C221C2B1C301C391CFBF7DFFF002295
:10AA80000B1C00920193101C3B1C321CFDF7B4F808
:10AA9000021C0B1C201C291CFDF7AEF80290039130
:10AAA0006DE500240021FFF711FC2B1C27492648E7
:10AAB000009AFCF7E7FA061C0D1CFFF72EFB304A44
:10AAC000304B04980599FCF705FE2D4A2D4BFCF7F9
:10AAD00001FE061C0D1CFFF720FB089E012E01D075
:10AAE000FFF765FB80200006051C069E6544FFF706
:10AAF00014FB002801D0FFF71FFB6346C91A221C74
:10AB00000A41101C8840A04201D0FFF7E5FA01235A
:10AB10001A4002239B1A0893FFF7DEFA1C4B994553
:10AB200000DDD1E5002398469946FAE58024E40249
:10AB30000121FFF7CBFB4A4600F006FA021C0B1C72
:10AB400099E66442A146DDE5000000000000F03F08
:10AB5000000000604715F73F44DF5DF80BAE543E40
:10AB6000000000000000D03F555555555555D53FC4
:10AB7000000000000000E03FFE822B654715F73F14
:10AB80009C7500883CE4377EFEFFEF3F0000F03FFD
:10AB90000000E03FC046C046F0B55F4656464D4611
:10ABA0004446F0B46C4E0D1C371C83B0041C021CD0
:10ABB0000B1C2F40B74200D1ADE0002900DC8BE038
:10ABC0002F1500D194E0654D09038023090B5B0329
:10ABD0007F190B43FE0700D570E07F10C20FB84607
:10ABE0005B00002780219B1816244200009700205C
:10ABF000890345189D4204DC68185B1B009D6D1895
:10AC00000095D50F5B00013C5B1952004908002CF0
:10AC1000EFD180210026090620250196B4468946F9
:10AC200009E0834246D0D40F5B00013D1B1952005E
:10AC30004908002D1CD066468C198342F1DD671847
:10AC4000E60FBC46F60782464E452CD01B1AA242A0
:10AC500080414042019F1B1A121B7F18D40F5B00DA
:10AC6000013D019750461B1952004908002DE2D1C1
:10AC7000134328D101984308009D394E6A10921958
:10AC8000ED0702D5802109060B4340460705B91898
:10AC90001C1C0D1C201C291C03B03CBC9046994672
:10ACA000A246AB46F0BDFF0FFF077E427E41B24693
:10ACB0008244CBE79442C2D9181CB4E7C20F5B00B0
:10ACC0009B18400089E7019901312FD0019C012395
:10ACD00023401B195B08CFE76B005B081A43D9D0F0
:10ACE000002700292BD1C10A153F40050029FAD0C1
:10ACF0008022520311421ED1002349000133114228
:10AD0000FBD001242022E41AD21A3F19041CD4409B
:10AD10002143984057E7201C291CFCF7DBFC221C30
:10AD20002B1CFBF78BFE041C0D1CB3E7009A0023C1
:10AD300001320092A0E7202201240023E5E7221C33
:10AD40002B1C201C291CFCF757FF021C0B1CFCF7BA
:10AD500099F9041C0D1C9DE70000F07F01FCFFFF2A
:10AD60000000E03F4B0059087047C0464800024BC6
:10AD70004008C018C00F7047000010800B1C011C59
:10AD8000021C30B519430220002900D130BD8021BA
:10AD900009068B4216D00D4904205C180C498C42E0
:10ADA000F4D90C4D5C198C42F0D90B4C5900490870
:10ADB0000320A142EAD9074C0020A142E6D150422B
:10ADC0005041E3E7002AE1D0EFE7C0460000F0FF82
:10ADD000FFFFDF7F0000F07FFFFF0F0000207047C4
:10ADE000024901487047C046000000000000F87F9B
:10ADF000F0B546464F46C0B4CA0F90464B004D4A88
:10AE00005B0D9E1883B0041C0D1C8C46071C132E72
:10AE10003BDC002E5CDB484F021C37413B1C0B40E7
:10AE20000343994648460B1C002827D07B081A1C70
:10AE30000A4022430027002A0AD0132E00D176E0D0
:10AE4000291C80229943D2020B1C324113439C4699
:10AE50004046C1003948634641180C684D683A1CA9
:10AE6000201C291CFBF7EAFD009001910098019934
:10AE7000221C2B1CFCF7C0FE021C0B1C101C191CF6
:10AE800003B00CBC90469946F0BD332E0BDD0B1C75
:10AE90008021021CC9008E42F0D1291CFBF7CEFD97
:10AEA000021C0B1CEAE7264A0126D2187642D6403D
:10AEB00091460B1C021C0642E0D076080642C7D021
:10AEC0008023B443DB0548460341271C1F43BFE7EB
:10AED0004E0076080643021C0B1C002ECED0090340
:10AEE000090B01434842014380200003090B014044
:10AEF000680C40040B1C03434046C1000F48411836
:10AF00000C684D68291C201CFBF798FD00900191EE
:10AF1000009801992B1C221CFCF76EFE0D1C41466B
:10AF2000021CC80769004908031C0B43A6E78027D9
:10AF30003F0685E701FCFFFFFFFF0F0098B402000A
:10AF4000EDFBFFFF00000000F8B53D4E171C331C61
:10AF50000B40041C0D1C0A1C1B1525D14B005B0863
:10AF600018431ED0201C291C2E4B2D4AFCF7B2FB87
:10AF7000344B041C0D1C9F4231DB0E4033150A1C60
:10AF8000363B3149DB198B4215DD221C2B1C264830
:10AF9000264900F061F8244A244BFCF79BFB041C73
:10AFA0000D1C291C201CF8BD28498B421ED02649A7
:10AFB000DB198B42E9DC002B05DD25491B050A4026
:10AFC0001D1C1543EDE7191C353118DA214B9F4242
:10AFD000DBDC17481749221C2B1C00F03DF8144AF3
:10AFE000144BFCF777FB041C0D1CDAE7201C291C12
:10AFF000221C2B1CFBF722FD041C0D1CD1E714495D
:10B0000036331B050A401D1C1543201C291C0A4A07
:10B010000A4BFCF75FFB041C0D1CC2E7C046C04690
:10B0200000000000000050439C7500883CE4377E1F
:10B0300059F3F8C21F6EA501000000000000903C0B
:10B040000000F07FB03CFFFFFE070000FF0700009C
:10B05000FFFF0F8050C3000030B5DA0FD2074B005E
:10B060005B08111C194330BD014B18687047C0467E
:10B0700060240020F8B5C046F8BC08BC9E46704766
:10B08000F8B5C046F8BC08BC9E46704743000000B7
:10B0900000240020181801000A1801002E2E2F622B
:10B0A0006C655F616E742E6300452D4D6F74696F22
:10B0B0006E00496E73696465205269646500256994
:10B0C0002E25692E2569002E2E2F6972745F7065FA
:10B0D000726970686572616C2E63002E2E2F6D612F
:10B0E000696E2E63002E2E2F2E2E2F6E7266353136
:10B0F0005F73646B2F496E636C7564652F6170704C
:10B100005F636F6D6D6F6E2F6170705F74696D65D9
:10B11000722E68002E2E2F2E2E2F6E726635315F06
:10B1200073646B2F496E636C7564652F73645F6322
:10B130006F6D6D6F6E2F736F66746465766963658E
:10B140005F68616E646C65722E68002E2E2F6C69CC
:10B15000627261726965732F626174746572792EAF
:10B1600063002E2E2F6C69627261726965732F6E97
:10B1700072665F70776D2E63002E2E2F6C6962727F
:10B1800061726965732F706F7765722E63002E2E62
:10B190002F6C69627261726965732F72657369736E
:10B1A00074616E63652E63002E2E2F6C696272616E
:10B1B000726965732F73706565642E6300B9A5218C
:10B1C000FBBD72C3452E2E2F73657276696365735E
:10B1D0002F616E745F62696B655F706F7765722E49
:10B1E00063002E2E2F73657276696365732F616E0F
:10B1F000745F62696B655F73706565642E630002DE
:10B2000000000000000010B9A521FBBD72C3452E4F
:10B210002E2F73657276696365732F616E745F6339
:10B2200074726C2E63008BEB9F0F50F1FA97B34A48
:10B230007D0A000026A02E2E2F7365727669636545
:10B24000732F626C655F6370732E63002E2E2F2E3A
:10B250002E2F6E726635315F73646B2F536F75726C
:10B2600063652F73645F636F6D6D6F6E2F736F66B1
:10B27000746465766963655F68616E646C65722E7F
:10B2800063002E2E2F2E2E2F6E726635315F736463
:10B290006B2F536F757263652F626C652F626C65DF
:10B2A0005F73657276696365732F626C655F64694D
:10B2B000732E63002E2E2F2E2E2F6E726635315F69
:10B2C00073646B2F536F757263652F6170705F636A
:10B2D0006F6D6D6F6E2F6170705F74696D65722E2A
:10B2E00063002E2E2F2E2E2F6E726635315F736403
:10B2F0006B2F536F757263652F6170705F636F6D35
:10B300006D6F6E2F6170705F7363686564756C65D7
:10B31000722E6300EE600200A2600200CE600200A6
:10B320002A600200CE600200C6600200CE60020009
:10B330002A600200A2600200A2600200C660020051
:10B340002A600200226002002260020022600200E5
:10B35000D4600200866402008064020080640200FF
:10B3600076640200D8630200D86302006E640200B3
:10B3700076640200D86302006E640200D8630200A3
:10B3800076640200D6630200D6630200D663020030
:10B390000E6502007472020008720200527202000E
:10B3A00036710200527202004472020052720200B0
:10B3B0003671020008720200087202004472020034
:10B3C000367102002C7102002C7102002C710200F7
:10B3D00098740200BC780200AA7A0200AA7A0200DD
:10B3E0009A78020082770200827702008A7802004F
:10B3F0009A780200827702008A780200827702003F
:10B400009A7802008077020080770200807702003D
:10B41000B27A0200232D302B2000686C4C00656648
:10B420006745464700303132333435363738394195
:10B4300042434445460030313233343536373839AB
:10B440006162636465660000666D6F640000000001
:10B45000706F770000000000000000000000000096
:10B46000000000000000008000000000000000005C
:10B470000000004003B8E23F0000000000000000B0
:10B4800006D0CF43EBFD4C3E000000000000F03F33
:10B49000000000000000F83F000000000000304302
:0CB4A00000000000000030C300000000AD
:08B4AC00144CFF7F01000000B9
:10B4B4000000000000000000000000000000000088
:10B4C4000000000000000000000000000000000078
:10B4D4008CB002000000000000000000000000002A
:10B4E4000000000000000000000000000000000058
:10B4F4000000000000000000000000000000000048
:10B504000000000000000000000000000000000037
:10B5140000240020FFFF0000630D0200550D02000F
:10B524004B0D02003D0D0200950C0200DD110200DE
:10B534005D14020001160200AD0C0200491602005F
:10B5440049110200351602009D150200890C020003
:10B55400F513020000FFFFFF0000000001000000DF
:04000003200001C513
:00000001FF
